:020000040001F9
:1000000008680020490301005B030100511601004C
:100010005F0301006103010063030100E070F9DF89
:100020008F9E939B06999697020100005D02010046
:1000300067030100ECB30100E50201003503010094
:100040006D0301006D0301006D0301006D030100EC
:100050006D0301006D0301006D0301006D030100DC
:10006000514D01006D0301006D0301006D0301009E
:100070006D0301006D0301006D0301006D030100BC
:100080006D0301006D0301006D0301006D030100AC
:100090006D0301006D030100092901006D030100DA
:1000A0006D0301006D0301006D0301006D0301008C
:1000B0006D0301006D0301006D0301006D0301007C
:1000C0006D0301006D030100292901002D290100A4
:1000D000312901006D0301006D0301006D03010072
:1000E0006D0301006D0301006D0301006D0301004C
:1000F0006D0301006D0301006D0301006D0301003C
:100100006D0301006D0301006D0301006D0301002B
:1001100000F002F800F05AF80AA090E8000C8244BF
:100120008344AAF10107DA4501D100F04FF8AFF29C
:10013000090EBAE80F0013F0010F18BFFB1A43F0C5
:100140000103184748CA000068CA00000A444FF07B
:10015000000C10F8013B13F0070408BF10F8014B26
:100160001D1108BF10F8015B641E05D010F8016B6B
:10017000641E01F8016BF9D113F0080F1EBF10F8CF
:10018000014BAD1C0C1B09D16D1E58BF01F801CBF2
:10019000FAD505E014F8016B01F8016B6D1EF9D575
:1001A0009142D6D37047000000230024002500268A
:1001B000103A28BF78C1FBD8520728BF30C148BFCA
:1001C0000B6070471FB51FBD10B510BD00F0D2FA0F
:1001D000114603B404F0A8FE03BCFFF7F3FF00F0E0
:1001E00001FB00F0ECFA03B4FFF7EEFF03BC00F0F4
:1001F000EFFA000080F309887047EFF30980704739
:10020000684680F3098804480078C00714BF0220BC
:10021000032080F31488704724BE0100DFF818C063
:10022000EFF305831B0618BF6047EFF31483DB076A
:1002300008BF604700DF704729790100DFF818C068
:10024000EFF305831B0618BF6047EFF31483DB074A
:1002500008BF604700DF7047357B0100EFF309807E
:10026000816911F8021C39BB90E80F10E047EFF3E9
:10027000098C194B93E80600914218D059B10CB47F
:100280004FF0010381F821302CE9F00FC1F824C0B0
:1002900007F0E4FE0CBC1A60D2F824C0BCE8F00FF2
:1002A00092F821308CF309881BB192F82000CCF829
:1002B00000006FF0020E704710B5084A12689142B4
:1002C00009D8074C54F8214090E80F10A047EFF3ED
:1002D000098C8CE80F0010BD58040020E0070100D5
:1002E000E007010007F0A6FD114B93E806009142DC
:1002F0001BD00CB44FF0000381F82130EFF3098CD0
:100300002CE9F00FC1F824C007F0A8FE0CBC1A605D
:10031000D2F824C0BCE8F00F8CF3098892F82130A1
:100320001BB192F82030CCF800306FF0020E70470D
:100330005804002007F054FFD6E7000006F046FE00
:1003400007F04EFFD0E700000C4880470C4880477C
:100350000C48004730BFFFF7FDFFFEE7FEE7FEE772
:10036000FEE7FEE7FEE7FEE7FEE7FEE7FEE700004A
:1003700005480649044A064B70470000211C01004D
:10038000952701001101010008660020086800207F
:100390000866002000487047A865002040EA010375
:1003A00010B59B070FD1042A0DD310C808C9121F1E
:1003B0009C42F8D020BA19BA884201D9012010BD58
:1003C0004FF0FF3010BD1AB1D30703D0521C07E025
:1003D000002010BD10F8013B11F8014B1B1B07D189
:1003E00010F8013B11F8014B1B1B01D1921EF1D1FA
:1003F000184610BD10B5431C02E010F8011B71B186
:100400008107FAD14FF0013202C88C1A8C4314EAEA
:10041000C211F9D0C01A0A0603D0C01E10BDC01AFE
:1004200010BD0A0401D0801E10BD0902FCD0401E80
:1004300010BD40EA010370B59B072ED14FF0013685
:10044000042A2AD308C810C99D1B9D43121F15EA10
:10045000C61517D0D8B2E1B2401A50EA056110D1E2
:1004600098B2A1B2401A50EA05410AD123F07F4068
:1004700024F07F41401A50EA052102D1180EA0EB6A
:10048000146070BDA342DBD018BA21BA884201D9EA
:10049000012070BD4FF0FF3070BD0AB9002070BD63
:1004A00010F8013B11F8014B63B1A3420AD1521E6F
:1004B00008D010F8013B11F8014B1BB1A34201D148
:1004C000521EEDD1181B70BD421E12F8013F002BC9
:1004D000FBD111F8013B002B02F8013BF9D1704729
:1004E000032A40F2308010F0030C00F0158011F860
:1004F000013BBCF1020F624498BF11F801CB00F838
:10050000013B38BF11F8013BA2F1040298BF00F88B
:1005100001CB38BF00F8013B11F0030300F0678006
:10052000083AC0F0088051F8043B083A51F804CB6F
:10053000A0E80810F5E7121D5CBF51F8043B40F835
:10054000043BAFF30080D20724BF11F8013B11F840
:1005500001CB48BF11F8012B24BF00F8013B00F884
:1005600001CB48BF00F8012B7047431A28BF9A42BD
:100570007FF6B6AF032A1044114440F2268010F0F3
:10058000030F1EBF11F8013D521E00F8013D10F08F
:10059000030F7FF4F6AF11F0030300F0C180083AB7
:1005A000C0F00B8051F8043D083A51F804CD40F8F2
:1005B000043D40F804CDFFF7F3BF121D5CBF51F8B6
:1005C000043D40F8043DAFF30080D20724BF11F88A
:1005D000013D11F801CD48BF11F8012C24BF00F8EE
:1005E000013D00F801CD48BF00F8012C704710B55F
:1005F000203AC0F00B80B1E81850203AA0E818501B
:10060000B1E81850A0E81850BFF4F5AF5FEA027CDB
:1006100024BFB1E81850A0E8185044BF18C918C04A
:10062000BDE810405FEA827C24BF51F8043B40F8EB
:10063000043B08BF7047D20728BF31F8023B48BFD0
:1006400011F8012B28BF20F8023B48BF00F8012B0E
:10065000704702F0FF0343EA032242EA024200F03D
:1006600002B84FF000020429C0F0128010F0030C11
:1006700000F01B80CCF1040CBCF1020F18BF00F895
:10068000012BA8BF20F8022BA1EB0C0100F00DB844
:100690005FEAC17C24BF00F8012B00F8012B48BFA2
:1006A00000F8012B70474FF0000200B51346944646
:1006B0009646203922BFA0E80C50A0E80C50B1F1BA
:1006C0002001BFF4F7AF090728BFA0E80C5048BFCE
:1006D0000CC05DF804EB890028BF40F8042B08BF6C
:1006E000704748BF20F8022B11F0804F18BF00F868
:1006F000012B7047704770477047431A28BF9A42D2
:100700007FF675AF104410F0030F11441EBF11F8AF
:10071000013D521E00F8013D10F0030F7FF4F6AFCB
:10072000103AC0F00A8010B531E91850103A20E9AB
:100730001850BFF4F9AFBDE81040530724BF31E9AA
:10074000081020E9081044BF51F8043D40F8043D6A
:1007500012F0030F08BF7047D20728BF31F8023DDF
:1007600048BF11F8012C28BF20F8023D48BF00F80F
:10077000012C70477546FFF70DFEAE460500694631
:10078000534620F00700854618B020B5FFF7F0FD6E
:10079000BDE820404FF000064FF000074FF0000882
:1007A0004FF0000B21F00701AC46ACE8C009ACE803
:1007B000C009ACE8C009ACE8C0098D46704710B567
:1007C0000446AFF300802046BDE81040FFF70BBDA4
:1007D00001491820ABBEFEE726000200704700006A
:1007E0000000000010B501F0ABFF00F004F8BDE818
:1007F000104006F06BB900207047000030B5224B66
:10080000186800F40062186840F4006018601E4820
:100810004C3001684904FCD41C48C16841F02001F7
:10082000C160C16841F40011C160174C18342168DF
:10083000856AC90A61F308058562416A41F00401CD
:100840004162416A41F001014162416A41F0100197
:100850004162C1688902FCD5416A21F0020141620E
:10086000C16821F02001C160416A2568C90D61F3AA
:10087000D32525601AB9196821F400611960416A0D
:1008800021F00101416230BD300A004000F001401A
:100890002DE9F04102787F2A03D0BDE8F04100F055
:1008A00089B801F8012B447801F8014B861C0D46EC
:1008B0004FF0021708E02946304600F07BF8074465
:1008C00006EB104615FA80F5641EF4D23846BDE8F2
:1008D000F081000070B500240B462246092841D063
:1008E0000ADC2D4A0928116953D2DFE800F0525280
:1008F00015181C23282E31004021FC2849D004DC87
:10090000F02835D0F12844D134E0FD2841D0FE282C
:100910003CD0FF283DD135E0184620A11CE01C4604
:1009200005F036FF21E00624224621491846FFF74C
:10093000D7FD2EE0184699B1D1F8A41103E018466E
:1009400071B1D1F8A81139B90AE01846D16FFAE7A8
:100950001846D2F88010F6E706F0CCFF044618E0FF
:10096000002416E00C4605F01BFF01462046F3E785
:1009700031200CE01970422058700F209870DA7006
:10098000042406E019705A70022402E00420187052
:100990000124204670BD0000ECB301004441504CDE
:1009A000696E6B20434D5349532D44415000000064
:1009B00070B401002DE9F8430278A2F180031F2BE7
:1009C00003D800F011F9BDE8F883A2F1A0035E2B73
:1009D00002D800F0A1F9F6E70A704C1C10F801CB20
:1009E00000250127FF217A4B7A4ADFF8EC914FF07E
:1009F0000116BCF11E0F70D2DFE80CF00F171E2A93
:100A00008F98B3E6CF303FE6E6E6E6E64347566624
:100A1000748A8DE6E6E6E6E6E6700078611CFFF78C
:100A200059FF207000F10210CDE7007818B30128BB
:100A300021D021701846B5E0057825B1012D03D0ED
:100A4000002525702EE00125177000F00DFFF8E756
:100A5000157000F035FE25703846A3E001885F4828
:100A60005F4A0068B0FBF2F00322801CB0FBF2F09A
:100A70004843401EFDD12570DCE7657025700220DB
:100A800090E0214600F09AFC8CE086780388C078DC
:100A900066F31F43534E53EA00603CD0906001F070
:100AA00031FECEE730467DE010F8016B0EB94FF411
:100AB00080760146304601F0EFFDF61D2570F00806
:100AC000000400F101106DE0007800F00301491C02
:100AD0001177C0F380005077B3E775E0214600F04E
:100AE0008BF95FE021700122144610F8013B0AE007
:100AF00010F8011B11F03F0100D14021C91DC908A8
:100B00000A440844521C5B1EF2D244EA024049E007
:100B100000782170D4E72170C4E701781174B0F82F
:100B200001109182B0F80300D0824BE01278214688
:100B3000012A13D00646401C10F8012B42B110F8D0
:100B4000013B9C0701D5DB0600D5001D521EF6D1E6
:100B5000801B0D7000044D70801C23E000F0CAF96A
:100B600020E0064610782146012809D00D704D700E
:100B7000A5700321F078800707D541F4802011E0AB
:100B8000304600F083FB0146F4E7B6F801004FF46D
:100B9000802202EB8040084304E01278012A04D04E
:100BA0002170484600F101100DE7C278B0F801103D
:100BB000007962F31F4141EA00600090694600201D
:100BC00001F006F92570ECE704F8011C3046FAE65E
:100BD000010002007C050020010005002003002028
:100BE00040420F00010004002DE9FC47027801F8A3
:100BF000012B0D464FF0011410F8011B0022670075
:100C0000803906464FF0010804F101090E2975D21A
:100C1000DFE801F007141F2E3C74747447535D62C3
:100C2000667705F0B5FD0646FFF7E4FBC4B22C700D
:100C3000681C22463146FFF753FC23E00724684630
:100C400002F016F8224669462846FFF749FC304C68
:100C500054E0684602F00CF830680090684602F0F4
:100C600027F8002002F09AF885F80080294C45E02A
:100C70003E21681C09F088F8040002D0012005F02C
:100C800039FF2C7004F58034A41C37E03778701CD1
:100C9000394609F0EFF8012005F02CFF85F80080B7
:100CA00028E085F80080307820B1012802D02A7031
:100CB0003C4623E006F0A0F8FAE785F8008004F04F
:100CC00099FA10B9022008F05BFD4C4616E0307826
:100CD00007F0DAFC2870EBE707F0A4FC2870F4E7D3
:100CE00016F8017B012005F015FF3946304607F064
:100CF0006DFD287004EB074404F101142046BDE8A3
:100D0000FC872A70307800B1012005F0B5FACFE7F2
:100D10000900010002000500FF2008704FF00110DB
:100D200070470000F0B52C4D2C492D4E2868DFF897
:100D3000B4C001EB800202F0704202EBC0103268D6
:100D4000002400EB82006044C0F80048264A106886
:100D500001EB800303F0704303EBC010234B1F68CB
:100D600000EB87006044C0F80048214C214F4FF051
:100D7000010E206801EB800101F0704101EBC01011
:100D8000396800EB81006044C0F800E82868134D22
:100D9000C03D05EB8000D0F880C031788E000F2177
:100DA00001FA06F62CEA060CC0F880C0106805EBC4
:100DB000800050F8802F1B789B0001FA03F39A43C0
:100DC0000260206805EB800050F8802F3B789B0084
:100DD00099408A430260F0BD10030020C0A000408B
:100DE0001403002000101402080300200C0300204C
:100DF000180300201C0300202DE9F05F002201F8F9
:100E0000012B012510F8019B8B46AA46044661E0A0
:100E100014F8017B17F03F0000D14020C01DC60828
:100E200038063048006825D52F4901EB8003D3F8F8
:100E300080C02E494FF00F0809688A0008FA02F8AE
:100E40002CEA080C4FF0040808FA02F84CEA080CE7
:100E5000C3F880C0244B0022C03303EB800303F0AF
:100E6000704303EBC01000EB810021490844C0F837
:100E700000280EE081001C48014451F8802F1B48D7
:100E80000F230078800083409A43052383401A4350
:100E90000A605A462146384600F02AFFB9F1000F91
:100EA00010D11048006881000F48014451F8802F8C
:100EB0000E480F230078800083409A430523834027
:100EC0001A430A60380602D5B344B24401E0344400
:100ED00035446D1CB9F101099AD24AEA0540BDE8D2
:100EE000F09F00000803002000A000400C03002039
:100EF000001014022DE9F04F87B005460590002040
:100F0000DFF880A3CDE901018C1C8AF80000039072
:100F10006978AD1C07465FEA010871D015F8016BCE
:100F2000B1076ED5F7B3DFF860B306F01100012802
:100F3000BBF8149007D0574669460E2000F048FFD2
:100F400002280ED013E06946304600F041FF022827
:100F50000ED1B9F1010903D39AF800100029F2D09B
:100F600040E1B9F1010902D339780029E4D0002722
:100F70000128F5D1009904F8011B0099090A04F829
:100F8000011B0099090C04F8021B0099090E04F8D2
:100F9000011C3FB131060ED5DBF80C1004F8011B23
:100FA0000A0A00E007E004F8012B0A0C04F8022BFF
:100FB000090E04F8011CF10652D5A97835F8030B87
:100FC00061F31F4015F8011B40EA01600490AE4830
:100FD000B0F816B0F00715D0AB48B0F81490002167
:100FE000304600F0F5FE022802D00128B8D109E011
:100FF000B9F10109B4D39AF800100029EFD0F1E05B
:1010000011E187E0A048B0F814906946304600F03E
:10101000DFFE022802D0012816D107E0B9F101094C
:1010200012D39AF800100029EFD00DE09649009AEB
:1010300089691140049A914206D0BBF1010B03D398
:101040009AF800100029DDD08F49009A8969114073
:10105000049A914201D040F01000012817D157E0C6
:10106000DFF824B2F107BBF8149022D007BB0021AF
:10107000304600F0ADFE022802D0012807D107E07B
:10108000B9F1010903D39AF800100029EFD0A9E0C3
:1010900031060CD5DBF80C1004F8011B0A0A04F821
:1010A000012B0A0C04F8022B090E04F8011C01277D
:1010B0002EE06946304600F08BFE022802D001285F
:1010C00007D107E0B9F1010903D39AF8001000290C
:1010D000EFD087E031060CD5DBF80C1004F8011BCB
:1010E0000A0A04F8012B0A0C04F8022B090E04F872
:1010F000011C009904F8011B0099090A04F8011B5E
:101100000099090C04F8021B0099090E04F8011C4F
:10111000002159E01FB35C48B0F8149069460E20D6
:1011200000F056FE022802D001285BD107E0B9F199
:10113000010957D39AF800100029EFD052E0009827
:1011400004F8010B0098000A04F8010B0098000C49
:1011500004F8020B0098000E04F8010C0027A9788F
:1011600035F8030B61F31F4015F8011B40EA0160DD
:101170000090B10603D544498861012025E0DFF8DD
:1011800008B1BBF814906946304600F021FE0228F1
:1011900002D0012826D107E0B9F1010922D39AF83B
:1011A00000100029EFD01DE031060CD5DBF80C1043
:1011B00004F8011B0A0A04F8012B0A0C04F8022B9C
:1011C000090E04F8011C012103910199491C0191A8
:1011D0009AF8001031B9A8F101015FEA01087FF423
:1011E0009DAE0CE0B8F1000F09D015F8011B8A077D
:1011F00001D5C90600D52D1DA8F10108F2E7012887
:1012000032D10FB320485746868A69460E2000F037
:10121000DFFD022802D0012826D105E0761E23D367
:1012200039780029F1D01FE0009904F8011B0099DA
:10123000090A04F8011B0099090C04F8021B009923
:10124000090E04F8011C0FE0039969B10E485746D6
:10125000868A00210E2000F0BBFD022804D1761EF4
:1012600002D339780029F4D0DDE901121170029916
:1012700048700298211A059807B0281A41EA0040E0
:10128000BDE8F08F000000207C0500202DE9F84F1C
:101290000026DFF82081054630468A46CF1C88F8B4
:1012A0000060B5F80140ED1C002C77D015F8019BCB
:1012B000DFF804B15FEA89715FD55FEAC97139D09F
:1012C000BBF814500021484600F082FD022802D0ED
:1012D000012863D12EE06D1E60D398F8001000291C
:1012E000F0D05BE024B95FEAC97001D04FF00E097D
:1012F000BBF814506946484600F06AFD022802D047
:1013000001284BD106E06D1E48D398F80010002943
:10131000F0D043E0009907F8011B0099090A07F88B
:10132000011B0099090C07F8021B0099090E07F828
:10133000011C761C641ED5D230E0A97835F8030B69
:1013400061F31F4015F8011B40EA016000901A4844
:10135000B0F814806946484600F03AFD022802D0F1
:1013600001281BD107E0B8F1010817D39BF8001042
:101370000029EFD012E0761C00E0C346641EDCD2E8
:101380000D485D46848A00210E2000F021FD0228D0
:1013900004D1641E02D329780029F4D08AF80060B1
:1013A000320A8AF801208AF80200A7EB0A00BDE899
:1013B000F88F0000000000207C0500202DE9F35F7D
:1013C0000578447802794188407962F31F4141EA07
:1013D0000066E0074FF001014FF0000807D02E48EB
:1013E000EA07006801D0016001E0C0F80080A007B2
:1013F00005D52A48AA0700D44146006801602006A6
:1014000003D52749E80909680860DFF898A0DFF8E4
:1014100098B0DFF8989066B32548864200D9064612
:1014200001F062FA0746E00704D0DAF8000000682D
:10143000A84219D1A00705D5DBF800000068B0EB81
:10144000550F11D1600702D5B8EB950F0CD1A0064E
:1014500002D5B8EB551F07D120060AD5D9F80000F0
:101460000068B0EBD51F04D001F03EFAC01BB042BB
:10147000D9D3DAF800000068DBF80010096840EA08
:101480004100D9F80010096840EAC11001990870BC
:101490000848BDE8FC9F0000F4020020FC02002088
:1014A00004030020F0020020F802002000030020C6
:1014B000C0C62D0001000600094910B500220A70BF
:1014C000084888600A7464238B82CA8201238A6177
:1014D0000B774A7701F016F9BDE81040FFF722BC00
:1014E0007C050020404B4C000078832805D08428E0
:1014F00003D08C2801D001207047002070472DE9CF
:10150000F0410446D0F808011E4615460F46002853
:1015100035D00846FFF7E8FF10B1012005F0F2FAD8
:10152000402D00DD4025D4F808012A46401EC4F8AD
:101530000801D4F81001394604EB8010FEF7D0FF03
:10154000D4F8100104EB80113846FFF7A1F9D4F864
:10155000101104EB4101A1F80001D4F8100104EBD3
:101560008010306094F81001401C00F00300C4F8B3
:101570001001D4F80C01401CC4F80C010120BDE896
:10158000F081D0F80C31E3B15B1EC0F80C31D0F81B
:10159000143100EB83130B60D0F8141100EB410100
:1015A000B1F80011116090F81411491C01F0030109
:1015B000C0F81411D0F80811491CC0F80811012016
:1015C0007047002070470022C0F810210421C0F8A5
:1015D0001421C0E94212704770B5054600F030F89A
:1015E0000028FBD1144C606A20F002006062A06801
:1015F00020F0704040F00050A060A06820F47F40D0
:1016000040F4AA40A0602560A06840F00400A060FB
:1016100000F016F80028FBD1A06808490840A06037
:10162000606A800705D5606A20F0020060620120D0
:1016300070BD002070BD000000200040FF00FF0FC3
:101640000248806800F0070070470000002000405A
:1016500003F0C0FB10B5FFF7F3FF08B1012010BD88
:101660000548016D41F000510165016D41F4805163
:101670000165002010BD0000002000401CB507F0EF
:1016800015FB00281BD09E208DF80000E7208DF868
:1016900001006946102000F0FFFF07F007FB00285B
:1016A0000DD000208DF800006946082000F0F4FFFE
:1016B00001A9002007F08EFA012800D000201CBDEF
:1016C000F0B52C4B2C49DFF8B8C01868002201EBAC
:1016D000800404F0704404EBC010284C256800EB33
:1016E00085006044C0F80028264D286801EB80067C
:1016F00006F0704606EBC010234E376800EB8700FB
:101700006044C0F80028214F386801EB800101F0E7
:10171000704101EBC0101E49D1F800E000EB8E00D3
:101720006044C0F800281868134BC03B03EB8000EE
:10173000D0F880C0227894000F2202FA04F42CEA38
:10174000040CC0F880C0286803EB800050F8804F7C
:101750003578AD0002FA05F5AC430460386803EB58
:10176000800050F8803F097889008A4093430360E5
:10177000F0BD000010030020C0A0004014030020B2
:1017800000101402080300200C030020180300209E
:101790001C030020F0B52C4B2C49DFF8B8C01868AA
:1017A000002201EB800404F0704404EBC010284CCC
:1017B000256800EB85006044C0F80028264D2868A5
:1017C00001EB800606F0704606EBC010234E37682A
:1017D00000EB87006044C0F80028214F386801EB17
:1017E000800101F0704101EBC0101E49D1F800E00A
:1017F00000EB8E006044C0F800281868134BC03B13
:1018000003EB8000D0F880C0227894000F2202FA07
:1018100004F42CEA040CC0F880C0286803EB8000B4
:1018200050F8804F3578AD0002FA05F5AC430460FE
:10183000386803EB800050F8803F097889008A40BF
:1018400093430360F0BD000010030020C0A00040DF
:101850001403002000101402080300200C030020D1
:10186000180300201C0300202DE9F04F6448016894
:10187000012201B90260634E634B306803EB8001C3
:1018800001F0704101EBC01060490C6800EB84006E
:101890005F4C2044C0F800285E4DDFF87CB128681A
:1018A00003EB800707F0704707EBC017DBF8000079
:1018B00007EB80002044C0F80028DFF860E1DEF884
:1018C000000003EB800707F0704707EBC017544890
:1018D000006807EB80002044C0F800284A4C3268BA
:1018E000C03C04EB820050F8807F0E684FF00F0C74
:1018F000B1000CFA01F827EA08074FF0050A0AFAC6
:1019000001F847EA08070760296804EB810081466F
:10191000D0F88070DBF80050A8000CFA00F827EA35
:1019200008070AFA00F847EA0807C9F88070DEF8E5
:10193000000004EB8007B946D7F88080384C246853
:10194000A7000CFA07FC28EA0C084FF0020C0CFA6E
:1019500007FC48EA0C08C9F880802B4FDFF8C490D8
:10196000C03707EB820C0CF0704C0CEBC21C0CEB7C
:10197000860808EB090CDFF8B080C8F800C003EB5C
:10198000820C0CF0704C0CEBC21202EB8606274A5C
:10199000DFF89CC01644CCF8006007EB810606F027
:1019A000704606EBC11606EB850C0CEB0906DFF85A
:1019B00084C0CCF8006003EB810606F0704606EBAD
:1019C000C11101EB85011C4D1144296007EB800119
:1019D00001F0704101EBC01101EB840505EB090139
:1019E000164D296003EB800101F0704101EBC0103E
:1019F000134900EB840010440860BDE8F08F00003C
:101A00005804004010030020C0A000401403002030
:101A100000101402080300200C030020180300200B
:101A20001C03002000301402F002002000181402F1
:101A3000F4020020F8020020FC0200200003002035
:101A4000040300202DE9F04F64480168012201B928
:101A50000260634E634B306803EB800101F070411C
:101A600001EBC01060490C6800EB84005F4C20441F
:101A7000C0F800285E4DDFF87CB1286803EB8007D2
:101A800007F0704707EBC017DBF8000007EB80009A
:101A90002044C0F80028DFF860E1DEF8000003EB26
:101AA000800707F0704707EBC0175448006807EB42
:101AB00080002044C0F800284A4C3268C03C04EB47
:101AC000820050F8807F0E684FF00F0CB1000CFAC6
:101AD00001F827EA08074FF0050A0AFA01F847EA71
:101AE00008070760296804EB81008146D0F8807000
:101AF000DBF80050A8000CFA00F827EA08070AFAF9
:101B000000F847EA0807C9F88070DEF8000004EB27
:101B10008007B946D7F88080384C2468A7000CFAB3
:101B200007FC28EA0C084FF0020C0CFA07FC48EA04
:101B30000C08C9F880802B4FDFF8C490C03707EB42
:101B4000820C0CF0704C0CEBC21C0CEB860808EB02
:101B5000090CDFF8B080C8F800C003EB820C0CF071
:101B6000704C0CEBC21202EB8606274ADFF89CC0D1
:101B70001644CCF8006007EB810606F0704606EBD1
:101B8000C11606EB850C0CEB0906DFF884C0CCF817
:101B9000006003EB810606F0704606EBC11101EB15
:101BA00085011C4D1144296007EB800101F0704153
:101BB00001EBC01101EB840505EB0901164D29600D
:101BC00003EB800101F0704101EBC010134900EB01
:101BD000840010440860BDE8F08F00005804004005
:101BE00010030020C0A000401403002000101402C5
:101BF000080300200C030020180300201C03002011
:101C000000301402F002002000181402F402002038
:101C1000F8020020FC020020000300200403002042
:101C2000094801220260094B1A600948D0F80011E6
:101C3000C903FBD5D0F8001141F00101C0F8001133
:101C40001A60002070470000040400400037004084
:101C5000003000402DE9F04107460C46154690073C
:101C600002D1FFF7EDFC10B10120BDE8F0811F4E5D
:101C7000B06820F0704040F00050B06010E0376075
:101C800001CD3063B06840F40030B060B06840F01F
:101C90000100B060FFF7D4FC0028FBD1241F3F1DDA
:101CA000042CECD29CB12B684FF0FF31FF2063EA8B
:101CB000000211400002641EF9D137603163B06840
:101CC00040F40030B060FFF7BBFC0028FBD1B068E7
:101CD00020F07040B060706A800704D5706A20F010
:101CE00002007062C0E70020BFE700000020004053
:101CF0002DE9F00710F03F0308BF402310F0800FDC
:101D00002F4DDFF8C0C04FF000094FF001062CD076
:101D1000002B12BFDFF8B0A0BDE8F0077047002429
:101D200008212F6811E0401EFDD1DAF80000D0F83C
:101D300000803E60DCF80400401EFDD1600840EAEF
:101D4000C814491EA3F1010306D0002B1CBFC7F81D
:101D50000090DCF80400E6D124FA01F002F8010B4F
:101D6000002BDCD1BDE8F0077047002B12BFDFF875
:101D70005C80BDE8F007704711F8012B082414E0DF
:101D8000D8F8007002F0010038602F68C7F80090A2
:101D9000DCF80400401EFDD13E60DCF80400401E6B
:101DA000FDD152085B1E641E04D0002BE8D1BDE8B3
:101DB000F0077047002BDFD1BDE8F0077047000047
:101DC000F40200207C050020F8020020FC02002024
:101DD000034A52780AB100F005B800F0D3B9000008
:101DE0007C0500202DE9F04FDFF870930123D9F82E
:101DF00000201360DFF868E34FF00008DEF80020F1
:101E0000C2F800801360D9F800C000F00102CCF8DD
:101E10000020DEF80020C2F800801360D9F80040EE
:101E2000420802F0010CC4F800C0DEF800C0CCF893
:101E30000080CCF8003000EB020CD9F8005082088A
:101E400002F001042C60DEF80040C4F8008023603A
:101E50009444D9F80050C20802F001042C60DEF866
:101E60000040C4F8008023606244D9F800C002F04A
:101E70000102CCF80020DEF80020C2F800801360D8
:101E8000D9F80020C2F80080DEF80020C2F80080F7
:101E90001360D9F800201360DEF80020C2F800803B
:101EA0001360B04A12684FEA820C0CF1804404F5CA
:101EB0002044D4F88060DFF8B0C20F27DCF800C0FF
:101EC0004FEA8C05AF40BE43042707FA05F53543BA
:101ED000C4F88050A54C04EB820404F0704404EB79
:101EE000C21202EB8C0202F1047202F58222C2F8E5
:101EF0000088DFF87CA29AF81C20002A18BFDEF8C0
:101F000000C005D0CCF80080CCF80030521EF9D1CA
:101F1000DEF80020C2F80080DFF858B2DBF800C01D
:101F2000DCF800C01360C2F80080DBF800402468D1
:101F300013604CEA440CC2F80080DBF800402468CF
:101F400013604CEA840CBCF1010F25D0BCF1020FE8
:101F500018BFBCF1040F7DD09AF81C00213004D0CA
:101F6000C2F800801360401EFAD17E4800688000ED
:101F700000F1804000F52040D0F880407A490F22DF
:101F8000097889008A409443052202FA01F121432D
:101F9000C0F8801000F0DBB810F0020F41D000262E
:101FA00035462024C2F80080DBF800703F681360DB
:101FB00076083D4446EAC776641EF3D1C2F8008035
:101FC000DBF800402468136085EA040212F0010F78
:101FD00018BF4FF0080C002918BF0E609AF81C10AB
:101FE000002918BFDEF8002005D000BFC2F800802D
:101FF0001360491EFAD15B490968890001F18041EB
:1020000001F52041D1F88050574A0F2412789200F0
:102010009440A543052404FA02F22A43C1F8802023
:1020200039E09AF81C4024B1C2F800801360641EA5
:10203000FAD14C4A1268920002F1804202F5204225
:10204000D2F88060484C0F252478A400A540AE4308
:10205000052500E03CE005FA04F43443C2F8804072
:102060000968002220247746D9F8006001F00105B4
:1020700035603D68C5F800802B600A444908641E3D
:10208000F2D102F00101D9F800201160DEF8001051
:10209000C1F800800B6010F0800F0AD03648374935
:1020A0000068B0FBF1F036494968B1FBF0F0CAF8BE
:1020B0000C009AF81000E0B3D9F80010C1F80080C5
:1020C000DEF80010C1F800800B60401EFAD13EE03F
:1020D0009AF81D1000291CBF10F0020F212104D016
:1020E000C2F800801360491EFAD19AF81C1021B181
:1020F000C2F800801360491EFAD11A4909688900A4
:1021000001F1804101F52041D1F88050164A0F2499
:10211000127892009440A543052404FA02F22A435F
:10212000C1F880209AF81D1019B110F0020F0ED1DD
:1021300000E00CE0D9F80000C0F80080DEF80010E4
:10214000212000BFC1F800800B60401EFAD1D9F8F1
:10215000000003600CF0FF00BDE8F08FFC020020DF
:10216000F4020020080300200C030020C0A000405F
:102170007C050020F80200202003002040420F00D0
:10218000001000E02DE9F04FFF4D002601232A68E2
:102190001360FE4CB44627683E60DFF8F4E3DEF8D7
:1021A0000420521EFDD13B60DEF80420521EFDD1FA
:1021B0002F6800F001023A602768C7F800C0DEF817
:1021C0000420521EFDD13B60DEF80420521EFDD1DA
:1021D0003718D5F80080460806F00102C8F800203C
:1021E000D4F80080C8F800C0DEF80420521EFDD1EB
:1021F000C8F80030DEF80420521EFDD13744D5F86F
:102200000080860806F00102C8F80020D4F800809B
:10221000C8F800C0DEF80420521EFDD1C8F8003016
:10222000DEF80420521EFDD13744D5F80080C608E0
:1022300006F00102C8F80020D4F80080C8F800C0F9
:10224000DEF80420521EFDD1C8F80030DEF804206C
:10225000521EFDD1BA192E6802F0010232602668C2
:10226000C6F800C0DEF80420521EFDD13360DEF84F
:102270000420521EFDD12A68C2F800C02668C6F8A4
:1022800000C0DEF80420521EFDD13360DEF80420C9
:10229000521EFDD1BC4A126813602568C5F800C003
:1022A000DEF80420521EFDD12B60DEF80420521E01
:1022B000FDD1B84A1268950005F1804606F5204622
:1022C000D6F88080B44D4FF00F092D68AF0009FAA1
:1022D00007F928EA09084FF0040909FA07F748EA5C
:1022E0000707C6F88070AD4E06EB820606F0704612
:1022F00006EBC21202EB850202F1047202F58222A1
:10230000C2F800C89EF81C50002D18BF26680CD0DB
:10231000C6F800C0DEF80420521EFDD13360DEF89E
:102320000420521EFDD16D1EF2D12268C2F800C0F9
:10233000DEF804506D1EFDD1DFF864B2DBF800500A
:102340002D681360DEF80460761EFDD1C2F800C06F
:10235000DEF80460761EFDD1DBF80060376813609C
:10236000DEF80460761EFDD145EA4706C2F800C0DB
:10237000DEF804506D1EFDD1DBF800502D681360AF
:10238000DEF80440641EFDD146EA8505012D2FD0FC
:10239000022D18BF042D00F01B819EF81C0010F1C7
:1023A00021010CD0C2F800C0DEF80400401EFDD1AF
:1023B0001360DEF80400401EFDD1491EF2D17548BD
:1023C0000068800000F1804000F52040D0F880C017
:1023D00071490F22097889008A402CEA020C0522F3
:1023E00002FA01F14CEA0101C0F8801000F045B991
:1023F00010F0020F5BD04FF00009C8462026F246CD
:10240000C2F800C0DAF80440641EFDD1DBF80040D9
:1024100027681360DAF80440641EFDD14FEA5904BE
:10242000B84444EAC779761EEAD1584EC2F800C0D3
:10243000DAF80440641EFDD1DBF800402468136024
:10244000DAF80420521EFDD188EA040212F0010FCE
:1024500018BF0825002918BFC1F800909AF81C2061
:10246000002A18BF34680CD0C4F800C0DAF8041091
:10247000491EFDD12360DAF80410491EFDD1521E19
:10248000F2D144490968890001F1804202F52042F5
:10249000D2F8806040490F24097889008C40A64317
:1024A000052404FA01F13143C2F8801055E09EF88A
:1024B0001C7074465FB100BFC2F800C06668761E2B
:1024C000FDD113606668761EFDD17F1EF4D1314ABE
:1024D0001268920002F1804202F52042D2F8808018
:1024E0002D4E0F273678B600B74028EA0708052793
:1024F00007FA06F648EA0606C2F880600026DFF80A
:1025000088A0DFF88890D1F800202027DAF8008032
:1025100002F00101C8F80010D9F80080C8F800C026
:102520006168491EFDD1C8F800306168491EFDD1BF
:10253000164452087F1EE9D1DAF8002006F00101A6
:102540001160D9F80020C2F800C06168491EFDD1B1
:102550001360DEF80410491EFDD110F0800F0AD080
:10256000104811490068B0FBF1F010494968B1FB0F
:10257000F0F0CEF80C009EF8101041B3024800684D
:10258000C0F800C0014813E0FC020020F402002063
:102590007C050020080300200C030020C0A00040A0
:1025A000F80200202003002040420F00001000E04D
:1025B000D0F80020C2F800C0DEF80400401EFDD1B3
:1025C0001360DEF80400401EFDD1491EF2D154E034
:1025D0009EF81D1000291CBF10F0020F21240CD002
:1025E000C2F800C0DEF80410491EFDD11360DEF809
:1025F0000410491EFDD1641EF2D19EF81C4064B146
:10260000C2F800C0DEF80410491EFDD11360DEF8E8
:102610000410491EFDD1641EF2D11B4909688900CE
:1026200001F1804101F52041D1F88060174A0F2463
:10263000127892009440A643052404FA02F2324331
:10264000C1F880209EF81D10B9B110F0020F14D10E
:102650000F480068C0F800C00E482121D0F80020C3
:10266000C2F800C0DEF80400401EFDD11360DEF8A1
:102670000400401EFDD1491EF2D1054800680360E8
:10268000E8B2BDE8F08F0000080300200C03002032
:10269000FC020020F40200202DE9F003451E3CBF9F
:1026A000BDE8F0037047DFF850900026DFF84CC01B
:1026B000134C012711F8012B5FF00803D9F8000033
:1026C00012F0010F14BF07600660DCF80080C8F844
:1026D00000606068401EFDD1C8F800706068401E50
:1026E000FDD152085B1E6D1E3CBFBDE8F003704774
:1026F000002BE3D1DEE70000FC020020F402002002
:102700007C0500200C490D4A0968B0EB910F02D3FB
:10271000012050700DE000EB5101491EB1FBF0F0BB
:1027200000235370022803D90321B0FBF1F000E02D
:102730000120506070470000200300207C0500202D
:102740000F4810B50068104983000E480B684FF021
:10275000010209D513F4401F0C4B03D00968C1F3E3
:10276000015108E0036010BD13F4E02F084BF9D0CD
:102770000968C1F302418A4093FBF2F1016010BD88
:10278000300A0040200300203C0A004000093D00C0
:1027900000D8B80510B472B6414942480160BFF391
:1027A0004F8F62B6404A9068810140480BD540493E
:1027B0004B6B5B1C07D08B6B5B1C04D04B6B041FFB
:1027C0002360896B06E001683A4B1940016001689B
:1027D00041F470210160106D37490843106533489A
:1027E0004838016841F01801016030482430016820
:1027F00041F006010160016821F0010101602B49EF
:1028000018390868820701F1040003D42B4A1268C2
:10281000520207D4026842F003020260026822F00A
:10282000030206E0026822F004020260026822F05D
:1028300020020260086840F0600008601B48183001
:10284000016841F00A010160016821F004010160A2
:10285000001D016821F00F01491C016013480C386C
:10286000016840F2014221F03F0111430160144828
:10287000016841F4805101600C482030016841F04A
:102880000101016007488030016841F47001016076
:10289000BFF34F8FBFF36F8F10BCFDF7AFBF0000CA
:1028A0000000010008ED00E000200040480A004060
:1028B00000100040FF07F0FF000001310008004059
:1028C00004040040BFF34F8F05480168054A01F436
:1028D000E06111430160BFF34F8F00BFFDE70000CF
:1028E0000CED00E00400FA05044805490068B0FB5F
:1028F000F1F004494968B1FBF0F070472003002073
:1029000040420F00001000E0064810B5016A016265
:1029100007F04EFD002803D0BDE8104000F004BAD7
:1029200010BD000000B0004000F004B800F002B894
:10293000AFF3008070B51B4D68684469446161065F
:1029400007D5016821F002010160016841F0020130
:102950000160200711D508266868C068C0060CD041
:10296000114802F075FB40B1A86890F800180E48B5
:1029700002F0D2FB68684661EEE7600705D470BDDF
:102980000A4802F08DFBA9680870084802F06DFB48
:102990000028F4D06868806800F01F002028EFD37A
:1029A00070BD000024030020DC470020CC3700204D
:1029B000002070470348D0E90410081A024909882A
:1029C000081A7047B804002022BC010070B50B4DF6
:1029D0000C460346D5E90C0188420BD9401A8442C3
:1029E00000DD044622461846FDF77AFD686B204458
:1029F000686300E00024204670BD0000B804002099
:102A0000002070472DE9F041194F0C460646D7E9E2
:102A10000401401A17490988081A002802DC00201E
:102A2000BDE8F081844200DD0446D7E906020025B6
:102A300090420FD3104B021919448A420AD30D1A3F
:102A400098462A463146FDF74BFD2E44641B40460E
:102A5000C7F8188034B122463146FDF741FDB86908
:102A60002044B8613969601901443961D8E7000030
:102A7000B804002022BC0100B659002010B5054C56
:102A80006068002805D10120606000F005F8002092
:102A9000606010BDB80400202DE9F047244CA06808
:102AA00000283ED0D4E90401421AE0684FF0000645
:102AB00052EA000137D021461E4FC969DFF87880FD
:102AC000DFF878901E4D7AB1A069814205D338882D
:102AD0008B182844834200D3421A99F8003038F802
:102AE0001300904200DA02461648E660007840F093
:102AF000800002F0EDF8E1690144E161626902449D
:102B000062613B882B448B4200D1E561216991428F
:102B10000BD199F8002038F81210814205D101201C
:102B2000E060BDE8F087A660FBE7E660F9E700003B
:102B3000B804002022BC010026BC01005B05002077
:102B4000B659002020BC010010B50B4C206A18B10A
:102B5000A06A401CA06210BD01202062606200F0EB
:102B60000DF8002060622062D4E90C018842F2D0A6
:102B7000401AFFF745FF10BDB804002010B5134CF4
:102B80001348164B216B0A1A12481B780088821AC8
:102B9000114830F8130082420EDB1148007801F032
:102BA000D3FC216B08442063A06A00280CD0616A22
:102BB000002909D1401E06E00120E062606A002879
:102BC00002D0A06A401CA06210BD0000B804002022
:102BD000F659002024BC010026BC01005B05002042
:102BE00021BC0100704700207047002070470000A2
:102BF00010B50B4800F03CF8002810D0084A0948EE
:102C0000116801700B0A43700B0C8370090EC170C0
:102C1000117901715179417191798171012010BD52
:102C2000F0040020B45800200E4810B50021416087
:102C30008160C1600C4A0161C0E90512C0E9072149
:102C400041620A4A8162C0E90B1242630180383056
:102C50004FF416520260017141710821817100F038
:102C600015F810BDB8040020B6590020F659002010
:102C700005490A6802600A7982714A794271897944
:102C800001710120704700003C01002010B506F0E2
:102C9000F5FF03F047FF012010BD10B507F07CF8E9
:102CA000012010BD10B507F0C5F8012010BD0000CF
:102CB000064902680A6082790A7142794A7100798C
:102CC00088710020C871084607F07CB83C010020DC
:102CD00010B510480024104944608460C460046149
:102CE000C0E90541C0E9071444620C498462C0E9A7
:102CF0000B4141630480FFF7D0FF06484FF41651A3
:102D0000383001600471447108218171FFF7D0FFF0
:102D100010BD0000B8040020B6590020F65900206C
:102D200010B5FFF7D5FF10BD70B519480078002821
:102D30002DD0184C00250126206A50B9D4E90C0189
:102D4000884206D11449884203D02163E562256296
:102D50006163A06A70B1206A60B9E06A50B9266206
:102D6000FFF70CFF2562D4E90C01884202D0401A1B
:102D7000FFF746FED4E90101084308D1D4E9040174
:102D8000884204D06660A660FFF786FE656070BD6D
:102D900059050020B8040020F659002070B570BD18
:102DA0000D480068C1698847A0B90C4C35B104F0E2
:102DB00041F82060002006F0E3FC0BE004F03AF854
:102DC0002168401AB0F5967F01D3012000E0002071
:102DD00003F0B0FE012070BDB4B80100380100203E
:102DE0000020704700207047024910B50880FFF7A7
:102DF00059FF10BDB80400200A4810B58278018838
:102E000062F31F41C27841EA026207490A6002790F
:102E10000A7142794A71807988710846FFF748FF44
:102E200010BD0000B4580020F004002010B5044686
:102E300001F0E6FE24F08000810004480844D0F848
:102E4000801221F48071C0F8801210BD0000104083
:102E500010B5817821F08001082912D2094C402256
:102E600004EB8103C3F8802282781306064A01D559
:102E7000022300E0012302F8213002EB8101808867
:102E8000488010BD00001040905E002070B50F4CCF
:102E9000B0B101252560002060600D480D49006833
:102EA000B0FBF1F04FF47A714843A060206A2062D1
:102EB000162001F081FF6562206840F4805002E036
:102EC000206820F48050206070BD000000B00040F9
:102ED0002003002040420F0000F00EBB1449A0B1B7
:102EE0004FF6FF70C1F80802D1F80C0240F4B85058
:102EF000C1F80C02D1F8800240F01000C1F8800245
:102F0000D1F8040240F402700FE0D1F80C0220F472
:102F1000B850C1F80C02D1F8800220F01000C1F8BE
:102F20008002D1F8040220F00800C1F804027047C2
:102F30000000104010B50B4C0B48A288007882426C
:102F400000D902461AB907490020143908718020B7
:102F5000216801F0BDFE216801442160A188081AA2
:102F6000A08010BD6C0500200BBC010010B5064C04
:102F70000020A288216801F0E7FA2168014421605D
:102F8000A188081AA08010BD6C05002070470000C1
:102F9000044A20F0800002EB80000021C0F880127B
:102FA000704700000000104070B5044603F0F6F9C9
:102FB000104D24F0800405EB8400D0F880220E49E7
:102FC00011F824301A4342F05002C0F8802211F860
:102FD000240001280CD1204603F0E0F9074901EB59
:102FE00084114160402101600120A040C5F82C02FD
:102FF00070BD000000001040905E0020905C00203A
:103000002DE9F0476E4F0446A7F1080580074FF001
:103010000009A5F1140622D501F038FE3878C00960
:10302000FFF7B4FFF888A8803878C0F3411121B1C8
:1030300001295AD002296FD165E07978DFF88481BF
:103040000C2969D2DFE801F0060C681368182768BC
:103050002B31384601F0ECFB1FE0FFF76BFF67E018
:10306000002005E001F022FED8F8000039E0012040
:1030700001F01CFCC0B3F5E710F01F0F4CD1B8787D
:10308000012140F08000307000F07F0001F0E7FD8A
:1030900001F00CFE4CE001F0CBFA28B3DDE710F0B4
:1030A0001F0F39D146481B3812E001F04FFCD8B150
:1030B00001F0FCFD444813E000F01F0001282BD173
:1030C000707888B13879B178884225D23F49084470
:1030D0002860C2E701F0FEFC30B101F0E7FD3C489A
:1030E000006828B3804723E016E010F01F0013D0DB
:1030F000012811D100F004F9D0B900F05DF9B8B998
:1031000000F0AEF807E010F01F0F05D100F082F9D3
:1031100070B900F0C3F958B93878000603D4F888BC
:1031200008B1002000E0802001F09AFDA5F804908D
:10313000600721D5387800061CD4A888E0B1FFF7D5
:1031400015FFA888C0B93878C0F3411161B10129D1
:103150000AD110F01F0007D0012805D100F062F855
:1031600050B900F037F838B9802001F079FDA5F8A2
:10317000049001E001F0A0FD200712D53878000688
:1031800006D5A888317908430BD0FFF7D3FE08E0B5
:103190003078010605D500F07F003070002101F085
:1031A0005EFD600602D50020FFF740FE200604D534
:1031B000BDE8F0478020FFF739BEBDE8F08700008A
:1031C0007405002084BC01007CBC01002B0400209D
:1031D00080BC010010B51049104A0879127890425D
:1031E00003D00F4A1278904214D1487820B10228B7
:1031F00005D020280ED10AE0FFF7F2FD02E0488852
:10320000FFF7F0FD30B101F051FD012010BDFFF7D7
:10321000F3FDF7E7002010BD740500203403002003
:103220003503002010B50B490B4A087912789042FB
:1032300003D00A4A1278904209D14878092806D169
:1032400000F0B4FA18B101F031FD012010BD0020EA
:1032500010BD000074050020370300203903002052
:1032600070B52249224A08791278904203D0214A47
:103270001278904237D11D4849781F4C1F4D408825
:1032800004291FD007DC79B101290FD002290BD006
:10329000032928D111E0202906D0212919D022297B
:1032A0001AD023291FD11AE02C6010E0FFF79DFCF3
:1032B00005E02C60FFF73EFE09E0FFF794FC0028D4
:1032C000F7D110E0FFF774FB0BE001F0EFFC0120F9
:1032D00070BDFFF78DFCF2E7FFF786FD01E0FFF719
:1032E0005DFD0028F1D1002070BD000074050020B4
:1032F0003403002035030020B45800206C05002062
:103300002DE9F041244E254930790978884203D0CF
:103310002349097888423CD17078224C224D234FB2
:103320000C2836D2DFE800F03506212C353535354E
:103330003516243100F0F6F958B3F078012802D0A0
:10334000032803D003E01A48206000E02560FFF75F
:10335000F1FD12E0F078022802D0032803D00CE03F
:103360001448206009E0256007E000F0C3F909E097
:1033700000F0F6F90BE001F099FC0120BDE8F081C6
:1033800000F0C6F928B12760E1E700F005FA00284F
:10339000F1D10020F2E7000074050020370300207F
:1033A000390300206C05002033040020B4580020AD
:1033B000F55800203659002010B51248124A0179FC
:1033C000127891421BD142784188C088FE2A09D0E8
:1033D000FF2A14D199B990B901F006F878B101F03B
:1033E00065FC0AE059B9012809D100F015FD30B19A
:1033F000074906480860FFF79DFD012010BD002029
:1034000010BD00007405002038030020B4580020CF
:103410006C05002070B51B4D1B49002668780978A3
:1034200088422CD1A888022829D1184CAA7812B336
:10343000002003E0217801B10C44401C411C8A4269
:10344000F8D82078B0B103F063F90146E01CFDF72D
:103450003BF80F4A012614602078E98881420BD995
:103460000C4990800978491E084206D10A4901207A
:10347000087002E0002602E09180FFF75BFD304615
:1034800070BD0000740500202ABC0100EC03002080
:103490006C0500200BBC01005C05002010B5104A33
:1034A0001049002450780978884217D1908807285D
:1034B00014D10E4B0C48012418600189D2888A422D
:1034C00009D90B4899800078401E014204D109496E
:1034D0000120087000E09A80FFF72CFD204610BD07
:1034E000740500202BBC01003E0300206C05002069
:1034F0000BBC01005C050020074800214170C16041
:1035000001614161418081808161C161C18001812E
:103510000162418170470000F80400202DE9F04766
:10352000494EB08871884A4FDFF820817D1C002405
:10353000884216D3B069A0B97461B4800123397888
:103540007A1C184606F040FF7080708848B1776199
:1035500098F80000012801D8756102E07088401CCD
:10356000708070884FF00109B0BBF06808B1F4605A
:1035700032E0316981B398F8000001280DD83C7021
:10358000B48002237A1C0021012006F01DFF708008
:10359000708800B1756134611EE03D78C846202D09
:1035A00000D3002508FA05F0084218D0681CC1B203
:1035B0003970B48002237A1C012006F005FF708068
:1035C000708818B177617088401C7080306908FA83
:1035D00005F820EA08003061708830B902E06D1CFF
:1035E000EDB2DCE7B069002829D07088B188DFF837
:1035F0006880401A85B2174F98F8000037F810001D
:10360000A84200D205461548007828B140F0800055
:103610002A46716901F05CFB7069114928447061A8
:10362000B088284480B2B0800988884209D298F8CE
:10363000000037F81000A84203D1C6F81890BDE882
:10364000F087B461FBE70000F804002012BC010021
:10365000F45800200EBC01005B0500200CBC0100EA
:1036600014BC0100F8B51C4C1C4D1D4F20890026D0
:1036700018B9E5613888E0802681E0882189421AFE
:103680001848E169007800F05FFF0004E169000C70
:103690000144E161218901448BB2238109D0398839
:1036A0008B4206D2114A1049127831F81210814229
:1036B00010D90F48017801200129009003D800217A
:1036C000064A022003E029786A1C02205B1E06F0ED
:1036D0000DFF2681F8BD0000F804002035590020B8
:1036E00016BC01000DBC01000EBC01005B050020F2
:1036F00013BC0100034804498078085C0349087042
:10370000012070477405002031040020B4580020C7
:1037100010B506F057FE02490870012010BD0000E8
:10372000B45800200B4910B5C8780022012804D0F5
:10373000022804D0032806D103E0074A02E0002053
:1037400010BD064A521C8978002306F03DFE012078
:1037500010BD000074050020F45800203204002041
:10376000094809498078C97810B1084A815409E0AC
:10377000084A0020064B127802E01954401CC0B2DF
:103780009042FAD3012070477405002030040020D5
:103790003104002012BC0100034810B5807806F007
:1037A000A3FE012010BD0000740500200C4908B5DF
:1037B000C8780022012804D0022804D0032806D1AA
:1037C00003E0002008BD074A00E0074A521C00231E
:1037D0000093CB88897806F089FE012008BD00009F
:1037E0007405002035590020320400202DE9F047EF
:1037F000DFF8DC80D8F80842C8F80842354D2007C9
:103800000FD5286828B1002028603348006800B12F
:10381000804704F04DF806F013FF3048006800B10F
:103820008047200601D504F043F8E0064FF0010779
:1038300004D52F602A48006800B18047294E6006F1
:1038400003D5316809B101208847A00603D5316846
:1038500009B100208847DFF89090E00505D56F603A
:10386000D9F8001009B102208847A00510D5D8F872
:103870003072C8F8307201260025374204D059F85A
:10388000251009B10820884776006D1C082DF4D357
:10389000600510D5D8F83472C8F8347201260025B6
:1038A000374204D059F8251009B104208847760022
:1038B0006D1C082DF4D3E00404D5D8F83C02C8F8F8
:1038C0003C02FEE7BDE8F047082001F075BA0000B1
:1038D000000010403404002038BC010030BC01005E
:1038E00034BC01002CBC01003CBC0100194810B5DF
:1038F000016841F0100101601748016841F01001B2
:1039000001601649086820F0407040F000700860BF
:10391000134C0020206001212160C4F80C024FF6F6
:10392000FF71C4F80812C4F80402D4F8041241F07C
:103930002001C4F80412C4F8040203F0B9FF0948D6
:10394000C4F82002E820C4F80C02BDE810400820AA
:1039500001F032BA00080040040400404005004075
:1039600000001040005C002070B500F005F9002850
:103970001CD00F4802220F4D027042700E4C0320E3
:103980002A632870A068022803D9A4F11F0082606E
:10399000A2600A480649007840F0800001F098F9DA
:1039A000A068296B401AA0600120207370BD000040
:1039B00076590020200500209B65002018BC0100DE
:1039C000114910B50878022808D0032810D004281F
:1039D00012D0052801D10020087010BD0B48C07B13
:1039E000282801D0A828F8D1BDE8104000F058BA26
:1039F000BDE8104000F030BD0548007840F0800080
:103A000000F042FDF4E70000200500207C65002066
:103A100018BC0100204A10B5117869B301290ED0F5
:103A20001E48052900781BD007292BD000F02CFD5B
:103A30001B4902200873BDE8104000F00DBD184876
:103A40001F38C07B2A2803D02F2805D0AA2822D1CE
:103A5000BDE8104000F0F8BABDE8104000F08ABAA6
:103A6000012181400F480068014201D0012000E09F
:103A7000002040F23F4200E009E0BDE810400AA10A
:103A800001F053BA00201070106B1F2803D1BDE85D
:103A9000104000F0C9B810BD2005002019BC01007D
:103AA0009B650020640500202E2E2F2E2E2F2E2EFB
:103AB0002F736F757263652F7573622F6D73632F2C
:103AC000757362645F6D73632E630000104910B5F7
:103AD0004868C86008B1012010BD0E4800F11F04FD
:103AE00082687AB1007B000604D50B48007840F06C
:103AF000800005E0A068096B884203D00748007881
:103B000000F0C2FC0120207300F0A6FC002010BDD4
:103B1000200500207C65002018BC010019BC0100B4
:103B20001048007900F08F01080605D501F00F005C
:103B30004FF48032824001E001228A400A48007836
:103B400040F0800088420CD108490968114208D031
:103B50000749084A0968914203D10D22044901F03E
:103B6000B7B870477405002018BC01006405002038
:103B70009B6500205553425370B50A48022400F15A
:103B80001F05816831B1007B000608D40648007823
:103B900000F07AFC2C7300F05FFC002070BD012067
:103BA00070BD00007C65002019BC010010B50E48F6
:103BB0000E4C8068216B884202D82063032000E00D
:103BC000042020700A480B49226B007840F08000E6
:103BD00001F07EF80448226B1F308168891A8160E9
:103BE0000021017310BD00007C650020200500202D
:103BF00018BC010076590020FFF7E2BE064810B558
:103C0000028807480549007800F09EFC05490863D2
:103C1000BDE81040FFF7FEBE1EBC01007659002033
:103C200019BC0100200500202DE9F047734E326BCE
:103C30001F2A01D2134600E01F230020704D714956
:103C400002E00C5C2C54401C9842FAD3DFF8BC9183
:103C50000127DFF8B4A199F800001F2A40F0800086
:103C60007ED129686A4A91427AD1654C69681F34CD
:103C70006160A968A160697B19B9A97B09B11029A4
:103C800001D927738AE0E97B4FF002082A293ED048
:103C900022DC1A294FD00FDC0429F2D006DCE9B36C
:103CA0000329EED1BDE8F04700F05CBB1229E8D152
:103CB000BDE8F04700F0B8B8232944D007DC1B2941
:103CC00035D01E29DDD1BDE8F04700F0DBB825294D
:103CD0003DD02829D5D148E09E2940D00FDC552978
:103CE000CFD004DC2F2954D03529CAD103E05A297A
:103CF00025D09129C5D1BDE8F04700F0F5BBA12939
:103D000029D0A3295DD0A8292FD0AA29B9D100F0A4
:103D100075FA002805D0287B000600E003E04BD4AC
:103D20003770BDE8F087BDE8F04700F0E5BBBDE8BF
:103D3000F04700F0BFBBBDE8F04700F037BABDE880
:103D4000F04700F007BABDE8F04700F0D5BABDE88B
:103D5000F04700F0A9BABDE8F047FFF705BE00E064
:103D600032E0BDE8F04700F051BB00F047FA002810
:103D7000D7D0287B000605D586F80080BDE8F0473F
:103D800000F08EB89AF8000000F07EFB84F80C80FA
:103D900004E0287C800705D400202073BDE8F047AC
:103DA00000F05ABB00F02AFA0028BAD0287B00069F
:103DB00002D437703762B4E799F8000040F0800011
:103DC000E2E700F061FB5CE74C4600F05DFB207829
:103DD000104C00F00F014FF48030884021685546A8
:103DE000084320609AF8000000F04EFB28788740D6
:103DF0002068074306202760307092E720050020E6
:103E00007C6500207659002019BC010018BC010017
:103E100055534243680500200249002008700120E4
:103E200070470000B458002010B5FFF7A5FE002829
:103E300020D0114B002080211870597002219970F8
:103E4000D97020241C7158719871D8710B48016881
:103E500008200A7812B11A54491C00E01C54401C76
:103E6000C0B22428F5D3064924200863BDE81040D9
:103E7000FFF79CBE10BD000076590020E80300202B
:103E8000200500200548C07CC107044800F11F0040
:103E900000D00121017300F0DFBA00007C65002032
:103EA0002DE9F0412E4D2F4F0026A969686ADFF8F1
:103EB000B88088420AD33878002440F0800000F0AF
:103EC000E3FA88F80C6000F0C7FA08E028492748B0
:103ED000097830F81140E86A844200D30446FFF7BD
:103EE000F5FD00B90024A86A48B374B1A96AE8696D
:103EF00022460144387840F0800000F0E9FEA86ACC
:103F00002044A862E86A001BE862D5E90410AA6AA6
:103F10004143914203D1AE62696A08446862D8F8AD
:103F200008104046091BC8F80810002C05D0E96AA3
:103F3000002902D1032129700673BDE8F081002C0D
:103F4000E3D0E96A28690144491EB1FBF0F26869CF
:103F5000824200D90246E969686A06F029FBC5E792
:103F60002005002018BC01009B6500201ABC010040
:103F70005B0500202DE9F0412F4C00252F4EA16953
:103F8000606A884207D32E482563007800F07CFAE7
:103F9000357300F061FAFFF799FD20B1206B08B38B
:103FA000A06A10B10FE0256320E0E16A20690144B6
:103FB000491EB1FBF0F26069824200D90246E16914
:103FC000606A06F0F5FA00201E49A36A226B0BE036
:103FD000D4F81CC01F181CF8077011F800C0674502
:103FE00001D0256202E0401C9042F1D3A16A206B0F
:103FF0000A18A262E16A0B1AE362D4E904714F4322
:10400000974203D1A562626A11446162B168091ADC
:10401000B16000280DD013B12078052809D1206A9D
:1040200028B100203073BDE8F04100F015BA01203E
:10403000F8E7BDE8F0810000200500209B65002026
:1040400019BC0100765900202DE9F041344D0026BD
:10405000344FA969686A884207D333482E630078D1
:1040600000F012FA3E7300F0F7F9FFF72FFD00B9E8
:104070002E63296BA86A08442969884206D9BDE8DD
:10408000F041FE2229A1002000F04FBF002030495E
:1040900005E0AB6AEC690A5C0344401CE2542A6BFD
:1040A0009042F6D3A86A11000844A862EA6AA2EB1B
:1040B0000102EA6222D092B988B129690844401EFF
:1040C000B0FBF1F46869844200D904462246E969EC
:1040D000686A06F087FAAE62686A20440DE0D5E9A6
:1040E000041202FB01F3834208D1E969686A06F011
:1040F00079FAAE626969686A08446862B968286BCF
:10410000091AB960002809D0E86A10B12878052892
:1041100004D13E73BDE8F04100F09EB9BDE8F081E6
:10412000200500209B65002019BC01002E2E2F2E9B
:104130002E2F2E2E2F736F757263652F7573622F5E
:104140006D73632F757362645F6D73632E6300001C
:104150007659002010B5FFF70FFD00281FD0FFF79C
:10416000B5FC00281BD00E480021062201700D4B23
:10417000427081701A7AD201C270017141718171ED
:10418000C1710949082018638A68082A03D9A1F176
:104190001F0290608860BDE81040FFF707BD10BDAA
:1041A00076590020200500209B65002010B5FFF700
:1041B000E3FC00281BD0FFF789FC002817D00C482F
:1041C0000321002201700B4942700B7ADB018370DE
:1041D000C2700420086308498A68042A03D9A1F13F
:1041E0001F0290608860BDE81040FFF7DFBC10BD83
:1041F00076590020200500209B65002070B5264CD4
:10420000264DB4F81100E17C40BA000440EA0121D7
:10421000207D01430020C5E90910E07B2F280AD04A
:1042200004DC28280BD02A2819D104E0A8280DD0B6
:10423000AA2814D106E0FFF749FC002829D0E08A1B
:1042400041BA0CE0FFF742FC002822D0B4F8150078
:10425000E17D40BA000440EA0121207E0143286943
:104260000D4E4143E962A06801251F3668B18842BE
:1042700010D0207B000604D50948007840F080006B
:1042800001E00848007800F0FFF8357300F0E4F82A
:10429000002070BD012070BD7C650020200500203D
:1042A00018BC010019BC010010B5FFF765FC00281F
:1042B0001CD0FFF70BFC002818D00D4A0D4891695F
:1042C000491E0B0E03700B0C43700B0A8370C170F8
:1042D00011690B0E03710B0C43710B0A8371C171D1
:1042E00008201063BDE81040FFF760BC10BD00005F
:1042F000200500207659002010B5FFF73DFC00286E
:1043000029D0FFF7E3FB002825D013480021134AEA
:104310000170417081700821C17091690B0E0371A9
:104320000B0C43710B0A8371C17102210172116977
:104330000B0C43720B0A8372C17209490C20106383
:104340008A680C2A03D9A1F11F0290608860BDE839
:104350001040FFF72BBC10BD76590020200500202F
:104360009B65002010B5FFF707FC002835D01B48DF
:1043700070211B4B017000214170DC685A6832EAE1
:10438000040406D006248470282404734173DA6080
:1043900008E0DAB1134A127BE2B1052282702022D2
:1043A00002734173C1700171417181710A22C2713E
:1043B000017241728172C1728173C173017441745F
:1043C00012201863BDE81040FFF7F0BB0222827094
:1043D0003A22E5E781700173E3E710BD76590020CA
:1043E000200500209B650020044900200860044946
:1043F0000860044907200870012070476805002004
:104400009B65002020050020FFF7EEBF10B5FFF7E9
:10441000B3FB002817D00C48202200210270417005
:104420000A4CC177032022632070094806490078AE
:1044300040F0800000F04CFC0648226B8168891A2D
:1044400081600121017310BD7659002020050020F4
:1044500018BC01009B650020084910B5064808609B
:1044600007480D22007840F0800000F031FC05493B
:104470000520087010BD0000555342539B65002075
:1044800018BC01002005002010B5044600F0E8FB30
:10449000200605D504F00F014FF48030884001E07C
:1044A0000120A04002490A681043086010BD0000C6
:1044B000640500200A4810B5817C00F11F0429B171
:1044C00001202073BDE81040FFF7C6BFC07C05493E
:1044D00000F00100486006F083F80020F1E70000DA
:1044E0007C65002020050020024900200873FFF7AA
:1044F000B3BF00009B6500200F4810B5816800F134
:104500001F0469B1007B000604D50C48007840F018
:10451000800001E00A480078FFF7B6FF012004E0C0
:10452000FFF7D4FA002805D000202073BDE8104022
:10453000FFF792BF10BD00007C65002018BC010091
:1045400019BC0100704700002DE9F04790460C4669
:10455000054601F023FF244ADFF89090064635F027
:1045600080074FF0010A28D12148416829B3082566
:10457000B8F1080F08D240F293121EA1002000F0FB
:10458000D4FC0020BDE8F08700214160D9F860022A
:1045900049462060D9F8640260602078000621D482
:1045A000E088F8B1D1F82C02C0071BD10E48903832
:1045B0004260E2880260504612E035684046A845F5
:1045C00000D2054602EB871188462A462046FBF7B3
:1045D00087FFC6F80480402030600AFA07F0494699
:1045E000C1F82C022846CDE7905C00200000104066
:1045F000340400202E2E2F2E2E2F2E2E2F736F756B
:104600007263652F6869635F68616C2F6D6178699B
:104610006D2F6D617833323632352F757362645F7A
:104620006D617833323632352E630000FFF778BA89
:104630002DE9FC414E4BA3F11C051878A3F10804A9
:1046400010F01F0002D001286DD179E04949D878D7
:10465000494E0A784649494F1C390628C97810D076
:1046600006DC012809D0022814D003287ED141E0BD
:1046700007282AD00F2879D156E04148206012201F
:104680005CE0002A72D019B13E4820600A2055E053
:104690003D48FAE70AB9012968D0022021B1009704
:1046A000787000209A7809E000967070F9E7009918
:1046B0000B7813B14B8819440091401C8242F6D10B
:1046C0000098017879B3206037E062B3072021B108
:1046D0000096707000209A7809E000977870F9E7EA
:1046E00000990B7813B14B8819440091401C824209
:1046F000F6D1E5E7254800909878032801D00020FE
:1047000008E002F049F80BE000990A780AB1114478
:104710000091401C99788142F6D10098017811B13E
:10472000206000780AE021E01948007800281BD0BA
:104730001848009020600178C1B14088019005E0E0
:1047400001A9684600F02AF800280DD0A188019838
:10475000814208D9104980B2A0800978491E0842D8
:1047600001D1012028710120BDE8FC810020FBE778
:104770007405002009BC0100EC570020360300201E
:10478000ACBC0100BFBC0100BEBC0100FABC010012
:104790000ABC0100C0BC01000BBC010070B5194A85
:1047A000194C1B4ED378194A2578212B1478154AB9
:1047B000127902D0222B22D116E0AA4201D0A242C5
:1047C0001DD1144A1378144A12780BB9012A16D055
:1047D00042B1124A02601046114A128810443060F9
:1047E000092009E00F4AF5E7AA4201D0A24206D10A
:1047F0000D4830600D4800880860012070BD002021
:1048000070BD00007405002037030020390300202C
:104810006C05002009BC01005B0500203603002068
:104820003C030020EC57002088BC0100AABC01001A
:1048300070B51C481B4C0078A4F1080410F01F0050
:104840000AD0184AA4F11403174D59781279012897
:1048500006D0022824D109E01248163820601DE055
:10486000F1B1987882421BD2002015E002F08F004F
:10487000020605D500F00F064FF48032B24001E089
:104880000122824009B900070AD19868104207D076
:10489000D868104000D0012028802560012070BD1C
:1048A000002070BD74050020B458002070B5264B60
:1048B000024619461878498810F01F00A3F11C061B
:1048C00004D0012829D0022827D111E0012924D1C0
:1048D00032B1012000F0FAF9F08840F0020005E062
:1048E000002000F0F3F9F08820F00200F08029E0C9
:1048F000187900F08F04200605D504F00F004FF45E
:104900008035854001E00125A540707828B1200759
:1049100003D0B068284200D009B1002070BD2AB190
:10492000204600F09DF9F06828430AE030692842EB
:1049300008D12046FEF77AFA2046FFF777FEF068A6
:10494000A843F060012070BD740500202DE9F05FE0
:104950005A480026017811F01F0F7DD1574F8078FB
:104960001C3FB1464FF0010A4FF4803B00287AD03B
:10497000534801783846C07809B901286CD008B18D
:10498000504C6CE0504C6AE06078022805D0042856
:1049900045D0052845D007285CD148486179807802
:1049A00081423AD1787020794949B8700020474A4D
:1049B000098802E002F80090401C8842FAD30125E1
:1049C000B8460AFA05F0D8F80810084202D028467E
:1049D000FEF7DEFAD8F808100BFA05F0084203D00B
:1049E00045F08000FEF7D4FA6D1C102DE9D34FF08E
:1049F0000110C8E902090120C8F81090FEF746FA34
:104A0000E0794006B8F8060002D540F0010001E068
:104A100020F00100A8F806001CE060881BE0E678A2
:104A200018E0BEB9A07800F08F05280604D505F07F
:104A30000F010BFA01F001E00AFA05F0B968014331
:104A40002046B960FEF704FA2846FEF7ADFA28467C
:104A500000F0D6F8207801E02BE004E00444207850
:104A6000002891D120E04D4687F8019001245E4650
:104A7000B9680AFA04F0084202D02046FEF788FA24
:104A8000B96806FA04F0084203D044F08000FEF74B
:104A90007FFA641C102CEBD34FF00110C7E902051C
:104AA00000203D61FEF7F2F9044879788078884269
:104AB00002D00020BDE8F09F0120FBE77405002034
:104AC00009BC010036030020EC5700202B04002015
:104AD0003A0300202DE9F84F444800273E4600786D
:104AE000BA4600F01F00B94601287CD13F491C3965
:104AF0004878002874D0002000903D48027808468D
:104B0000C0780AB901286ED08B4608B1394C63E0F1
:104B1000394C61E06078022805D004280AD00528C5
:104B20001AD0072856D161799BF80100814251D0F3
:104B3000608850E02D48A778E67801794FF00009A9
:104B4000B94247D18078B04244D1012000902B482F
:104B500010F807A0C6553DE024490879B84239D17C
:104B6000A07800F08F085FEA086005D508F00F0014
:104B70004FF48035854002E0012505FA08F5887874
:104B8000B04215D1DBF8081020462943CBF80810B5
:104B9000DBF80C10A943CBF80C10FEF759F940468E
:104BA000FEF702FA404600F02BF849EA050911E049
:104BB00056450FD119EA050F0CD1DBF80810404615
:104BC000A943CBF80810DBF80C10A943CBF80C1064
:104BD000FEF7DEF920780444207800289AD1009866
:104BE000BDE8F88FFFE70020FAE700007405002019
:104BF00009BC010036030020EC5700202B040020E4
:104C000070B5044601F0CAFB0E4D24F0800405EB9C
:104C10008400D0F8801241F04001C0F880120A48A8
:104C200010F8240001280CD1204601F0B7FB0749F9
:104C300001EB84114160402101600120A040C5F8D2
:104C40002C0270BD00001040905E0020905C00209F
:104C500010B5FEF765F8BDE81040FFF7D5BB70470B
:104C6000094930F0800008D001EB8000D0F88012B4
:104C700041F48071C0F880127047D1F8800240F48E
:104C80004070C1F8800270470000104008220249BD
:104C90000020FFF759BC00007405002002484FF4C3
:104CA0000071006902F0EEB80401002000221146F4
:104CB000802000F00DB8000002480349027800206F
:104CC000FFF742BC0BBC0100B45800207047000045
:104CD0002DE9F04714468946054601F05FFB194F60
:104CE000064625F080000122D7F8281202FA00F5C6
:104CF000294222D170B9D7F8801241F48061C7F8F7
:104D00008012114914B1402C19D001E08A68A2B177
:104D100000228A60402C00D940240C49224601EB35
:104D2000801080464946FBF7DBFBC6F80480346000
:104D3000C7F828522046BDE8F0870020FBE78A60CC
:104D4000EBE700000000104034040020905C0020DD
:104D50004FF0E0214FF48070C1F88001BFF34F8F16
:104D6000BFF36F8FFFF79ABF0348816821F070414E
:104D700081600020704700000020004000280DDB0B
:104D800000F01F02012191404009800000F1E02065
:104D9000C0F88011BFF34F8FBFF36F8F70470028AB
:104DA00009DB00F01F02012191404009800000F161
:104DB000E020C0F800117047002809DB00F01F0256
:104DC000012191404009800000F1E020C0F800116D
:104DD00070470000EFF3088400F00F010D2901D1A6
:104DE000EFF30984A18B04F12005890500D52D1D61
:104DF000C10600D4483500F069FAEFF3098000F0ED
:104E000065FAEFF3088000F061FAEFF3148000F028
:104E10005DFA284600F05AFA606900F057FAA06976
:104E200000F054FAE06900F051FA1248006800F00E
:104E30004DFA1048001F006800F048FA0D48001DA8
:104E4000006800F043FA0B481030006800F03EFAAA
:104E500008480830006800F039FA06480C3000684D
:104E600000F034FA432204A1002000F05EF8FDF7C0
:104E700029FDFEE72CED00E02E2E2F2E2E2F2E2EBC
:104E80002F736F757263652F6461706C696E6B2F21
:104E9000486172644661756C745F48616E646C65EC
:104EA000722E630010B5002A06DA22F00042D21DED
:104EB00022F00703102203E0D21C22F003030C228D
:104EC00013B19C188C4201D9012010BD0244014449
:104ED0008360C0E90021C91AD018884202D8106046
:104EE0000246F9E70020106010BD000010B504462E
:104EF00003F010FA002805D04FF6FF71DFF808C064
:104F0000206800DF10BD0000CD7D010010B5044613
:104F100003F000FA002803D0DFF808C0206800DFA3
:104F200010BD00001D7D010070472DE9F0411646BF
:104F30000F46002818D1EFF3108572B600231A46E9
:104F40001946184600F0E2F9040003D1314638460C
:104F500000F038FA85F31088002C05D1EFF30380B8
:104F6000C00601D105F084FEBDE8F08170477047AE
:104F700000207047704770477047000010B5282226
:104F80000D490E48FBF733FB05F034FF0C4805F0E4
:104F90002BFF05F05BFD0B490B4A0C4B08604FF4EF
:104FA0000071B0FBF1F01160094901221A6008603C
:104FB00009490848086010BDA0B40100F82C002081
:104FC00075590100540500203005002034050020EB
:104FD00038050020F82A00203C05002000B591B0DB
:104FE000FDF7E8FC402801D9402000E060B181B223
:104FF000684604F0C9FE010006D06846FDF702FDD0
:1050000010B1012001F076FD04F068FF0146402850
:1050100001D9402100E059B16846FDF7D7FC38B10D
:1050200081B2684604F026FF10B1012001F062FD54
:1050300001F078FD11B000BD0448417880788142CC
:1050400001D0012070470020704700008C00002034
:1050500030B50546EFF3108472B600F006F8A96883
:10506000081A84F31088401E30BDEFF3108372B627
:10507000D0E900128A4201D3501A02E0806810443D
:10508000401A83F310887047EFF3108372B6C0E9BB
:1050900002210021016083F3108841607047000005
:1050A00070B50446EFF3108572B6D4E9000188426A
:1050B00001D0012000E0002042220EA1FFF735FFC1
:1050C000E16820680E5C401C2060A16888420CD317
:1050D00002D14FF0010001E04FF000004FF0470215
:1050E00004A1FFF722FF0020206085F310883046DE
:1050F00070BD00002E2E2F2E2E2F2E2E2F736F758B
:105100007263652F6461706C696E6B2F6369726383
:105110005F6275662E63000070B50446EFF310857C
:1051200072B6C068626881546068401C6060A168A3
:1051300088420CD302D14FF0010001E04FF0000093
:105140004FF0300209A1FFF7F0FE00206060D4E9C3
:105150000001884201D0012000E00020352203A197
:10516000FFF7E3FE85F3108870BD00002E2E2F2E72
:105170002E2F2E2E2F736F757263652F6461706CE6
:10518000696E6B2F636972635F6275662E630000E0
:105190002DE9F04114460E460746FFF766FF8442AC
:1051A00000D220460546002404E03846FFF778FF89
:1051B0003055641CAC42F8D32846BDE8F0812DE997
:1051C000F04114460E460746FFF742FF844200D2E4
:1051D00020460546002404E0315D3846FFF79CFF79
:1051E000641CAC42F8D32846BDE8F08100F0B0BCA6
:1051F00000F0AEBC02488079002800D00120704742
:10520000BF3700200248C079002800D00120704735
:10521000BF3700200248407A002800D001207047A4
:10522000BF3700200248007A002800D001207047D4
:10523000BF3700202DE9F0418E212148FBF711FAFC
:10524000204C214F8E2520681D4EB84210D1A588D4
:105250008E2D01D22A4601E04FF08E0201D84FF088
:105260008E0518491648FBF73BF9002086F84700E1
:105270008E211448FBF7F5F92760A58041223546B9
:10528000F11DE01DFBF72CF935F8480F24F8480F05
:10529000A878A070E878E0708200094909484C318C
:1052A0004C30FBF71DF995F8440084F8440095F85C
:1052B000450084F84500BDE8F04100F0BFB80000AB
:1052C0003137002000000220646C766B074A92F8A8
:1052D0004B10102901D30020704702EB8101C864F4
:1052E00012F84B0F401CC0B2107070470000022033
:1052F00010B5054C4121E01DFBF7B3F9002024F85F
:10530000480FE07010BD0000000002202DE9F047BA
:10531000184F81461D4616468846F81DFBF76AF869
:10532000441CB9F1000002D04146FBF79AF9002075
:1053300006B1308005B12870F879002818D04445AE
:1053400002D8F91D224604E0A4EB0800C119424628
:10535000C91DB9F1000F02D0B7F84800308016B16E
:105360004846FBF7BDF815B197F84A0028700120B0
:10537000BDE8F08700000220014890F88C007047DB
:1053800000000220054A92F84B1029B102F14C01AD
:10539000016092F84B007047002070470000022027
:1053A00002488079002800D00120704700000220C8
:1053B000034890F88D00002800D0012070470000BD
:1053C000000002202DE9F04188460746FBF712F85D
:1053D000104D441C41263146E81DFBF742F9412C93
:1053E00002D83946224602E0413CE11932462C46B9
:1053F000E81DFBF775F8A4F8488000F009F908B13A
:10540000012003E000F006F900B1022084F84A0010
:10541000BDE8F08100000220014981F88C0070474E
:10542000000002200149887170470000000002203E
:10543000014981F88D0070470000022070B50022FC
:1054400011461046FCF706F91848174C0168216010
:1054500041686160008920810A21154800F006FE3C
:10546000144E134D60B12868B04209D1A8880A28AB
:1054700001D2AA8800E00A220D490B48FBF730F858
:105480000A202660A0800146094800F0EFFD28B1FF
:105490002868B04202D1A8880A2804D2BDE870402A
:1054A000014801F0D1BE70BDBF370020B8B801007F
:1054B00000E00700646C766B02498871084601F0D1
:1054C000C3BE0000BF3700200249C871084601F082
:1054D000BBBE0000BF37002002494872084601F0F9
:1054E000B3BE0000BF37002002490872084601F031
:1054F000ABBE0000BF3700202DE9F0410F46064645
:105500004FF0FF340025DFF83C8012E0705D082189
:1055100002F0A2F984EA006408204146002C02DA75
:1055200081EA440400E06400401E10F0FF00F5D161
:105530006D1CBD42EADB2021204602F08DF9C043FC
:10554000BDE8F081B71DC1042DE9F0410E461746B4
:105550002021C04302F080F904460025DFF83C809A
:1055600012E0705D082102F077F984EA00640820F7
:105570004146002C02DA81EA440400E06400401E47
:1055800010F0FF00F5D16D1CBD42EADB2021204662
:1055900002F062F9C043BDE8F0810000B71DC1040C
:1055A00070B514460D460646202A07D240F2DD1299
:1055B00009A10020FFF7B9FC022070BD00F018FD22
:1055C00008B1102070BD2A462146304600F0A8FEE2
:1055D0000028F7D0202070BD2E2E2F2E2E2F2E2EFD
:1055E0002F736F757263652F6461706C696E6B2FBA
:1055F000647261672D6E2D64726F702F6961705FC8
:10560000666C6173685F696E74662E6300000000EB
:10561000002070470120704710B500231A4600F0A3
:10562000CFFA002800D0012010BD10B505F02CF9EC
:10563000012800D0002010BD2DE9F041144E0024B7
:105640004FF460453078012806D040F2371211A19E
:105650000020FFF76AFC09E0B078022748B140F269
:105660003D120CA10020FFF760FC37700220BDE85E
:10567000F081204600F02AF810B137702220F6E7BA
:1056800004F50054AC42F4D30120B0700020EEE7E2
:10569000600000202E2E2F2E2E2F2E2E2F736F7592
:1056A0007263652F6461706C696E6B2F64726167E1
:1056B0002D6E2D64726F702F6961705F666C6173FF
:1056C000685F696E74662E630000000070B5214E3D
:1056D00004463078012805D0FF221FA10020FFF7E3
:1056E00024FC18E04FF40050B4FBF0F100FB114132
:1056F000022511B140F2071208E0F17869B1D6E94C
:1057000002121144A14208D04FF4877212A1002066
:10571000FFF70BFC3570022070BD4FF4FC22B4F58E
:10572000803F01D3944211D30121F170C6E90240B8
:10573000204601F077F9262803D00028ECD03570F8
:1057400070BD204600F054FC0028F9D035702120AF
:1057500070BD0000600000202E2E2F2E2E2F2E2E2A
:105760002F736F757263652F6461706C696E6B2F38
:10577000647261672D6E2D64726F702F6961705F46
:10578000666C6173685F696E74662E63000000006A
:105790004FF400507047000010B5282804D2064985
:1057A00051F82000002805D1F72204A10020FFF7BE
:1057B000BCFB0AA010BD0000E4B701002E2E2F2E66
:1057C0002E2F2E2E2F736F757263652F6461706C90
:1057D000696E6B2F6572726F722E6300000000009D
:1057E00001460120282901D20148405C7047000091
:1057F000BC0000202DE9F04789460446804600E0C1
:10580000641C2078402802D00028F9D163E0607839
:10581000622847D012DC522853D008DC422841D0FD
:10582000442848D0482840D04D2817D133E0542888
:105830003ED0552832D0562810D13FE0722840D0B3
:1058400006DC642837D068282FD06D2806D122E0E6
:1058500074282DD0752821D076282FD020A5204659
:10586000FAF7C8FD07462846FAF7C4FD0646A01910
:10587000C11908EB0902891E91422BD2BA1EA11C44
:10588000FAF773FE324629462046FAF729FE2078B9
:105890000028B6D11FE000F073FF01E000F078FFB0
:1058A0000546DCE700F034FFFAE700F065FFF7E7B4
:1058B00000F06AFFF4E700F05BFFF1E700F070FF33
:1058C000EEE7094890F82A0010B1074D2A35C6E7DF
:1058D00006A5C4E73C44A4EB0800BDE8F08700003F
:1058E0004552524F52000000ECB3010068747470CE
:1058F000733A2F2F6D6265642E6F72672F64657621
:105900006963652F3F636F64653D40553F766572FF
:1059100073696F6E3D40563F7461726765745F696D
:10592000643D4054000000002DE9F043A3B08846D8
:1059300081461E461746802102A82A9DFAF7B3FE2B
:10594000002002AC03E02154401C7F2802D2295CD5
:105950000029F8D180212046FFF74CFFCDE9004017
:1059600033463A464146484604F0C4FE23B0BDE8FB
:10597000F08370472DE9F0411E4615460C46074658
:1059800005F0E2FA2C4890F8201003290FD0022CE1
:105990000FD004B3012C0AD10168A94207D190F8B5
:1059A0002210A9B300214A1E016082608161BDE816
:1059B000F0810068A842FAD1304605F02DF804467F
:1059C000304605F02BF80646384602F0E7FE03465F
:1059D0002246314617E0384602F0E0FE0328E6D0C2
:1059E000304605F017F88007E1D4384602F0D6FEBD
:1059F0000746304605F010F80446304605F00EF82C
:105A000001463B4622462846BDE8F04104F034B842
:105A100028220A490848FAF7EAFD03F0AFFC0848D3
:105A20008178012903D14178022900D18170BDE834
:105A3000F04103F0ABBC0000F82C0020A0B4010042
:105A40008C0000202DE9F0411D4E0446174696F8C3
:105A500022008846550260B92946404602F05AFEA7
:105A6000032802D0214603F0B1FF96F82200002857
:105A70000FD07068A0420CD8F068A0420BD008D9B3
:105A80003069401C00D134613069A04200D2044624
:105A90003461BDE8F081F0692A461044F061E019F4
:105AA000F06096F8230020B1BDE8F041002004F03A
:105AB00033B841462046BDE8F04103F023BF000063
:105AC000F82C0020F0B518A185B00968049102787F
:105AD000002104AB5C5C944224D0491C0329F9D317
:105AE00012A1002291E878006F46815C8DE8780071
:105AF000A1F1610CBCF1190F14D9202901D205299B
:105B000010D14FF0000C17F80CE08E450AD00CF1C4
:105B1000010CBCF1100FF6D3521C0B2AE5D3012067
:105B200005B0F0BD0020FBE7E5002000222A2B2C69
:105B30002E2F3A3B3C3D3E3F5B5C5D7C0348006959
:105B400008B1012070470020FCE70000ECB3010021
:105B500070B50D4D00202C7874B100212970A97802
:105B600009B100F093FB022C05D06978032902D01B
:105B7000002800D1252070BD40F26B1203A1002047
:105B8000FFF7D3F9022070BD300000202E2E2F2EFB
:105B90002E2F2E2E2F736F757263652F6461706CBC
:105BA000696E6B2F647261672D6E2D64726F702F3A
:105BB000666C6173685F6465636F6465722E630011
:105BC00070B51C460546302901D3012000E00020B5
:105BD000472212A1FFF7A9F9286A696A1C4E0CB97D
:105BE000002232711B4A91420AD11B49884201D1DD
:105BF000022070BD1849FC3988420CD1012070BDCB
:105C0000284604F0F1FD18B11CB90120307100E004
:105C10000CB1032070BD002070BD00002E2E2F2E71
:105C20002E2F2E2E2F736F757263652F6461706C2B
:105C3000696E6B2F647261672D6E2D64726F702FA9
:105C4000666C6173685F6465636F6465722E630080
:105C500030000020069996978F9E939B2DE9F05F68
:105C60004FF00004DDF828B05FEA030891468A4649
:105C70000746254612D05FEA0B000FD00020C8F877
:105C800000000646CBF80000FFF7C2FC88B14FF4D5
:105C90008030022F06D0032F04D030E0712241E083
:105CA000064616E0B9F1000FFAD08245F8D01B2461
:105CB00026E0FFF7AFFC10B3012F02D0032F0AD06C
:105CC0001DE0B9F1000F04D0BAF1000F01D01A2481
:105CD00016E017480FE01748006980B10C3003E068
:105CE0008168012909D0143001680029F8D1416880
:105CF0000029F5D11048056802E00668FAE71C247F
:105D0000FFF780FA08B9012F03D024B12046BDE87F
:105D1000F09F1C24FAE725B1C8F80060CBF80050CA
:105D2000F4E7B82205A10020FFF7FFF80220EEE714
:105D30009CB40100ECB30100B4B801002E2E2F2E4C
:105D40002E2F2E2E2F736F757263652F6461706C0A
:105D5000696E6B2F647261672D6E2D64726F702F88
:105D6000666C6173685F6465636F6465722E63005F
:105D700030B5164C00236178012904D0022905D0E2
:105D8000032921D105E04FF4604318E04FF4FC23D0
:105D900015E02179C1B10E490969A9B10C3107E0BB
:105DA000844204D84C68844201D34B6806E0143125
:105DB0000C68002CF4D14D68002DF1D123B11044B2
:105DC000984201D3012030BD002030BD30000020BA
:105DD000ECB3010010B50C4C207830B1DA220BA1E5
:105DE0000020FFF7A2F8022010BDFF223021144846
:105DF000FAF72FFC0120207000206070A060E060A6
:105E00002061A070E07010BD300000202E2E2F2EDB
:105E10002E2F2E2E2F736F757263652F6461706C39
:105E2000696E6B2F647261672D6E2D64726F702FB7
:105E3000666C6173685F6465636F6465722E63008E
:105E4000A00600202DE9F04116460F460546002425
:105E5000FFF7E0FB50B1032D08D10648006928B1D7
:105E600031463846FFF784F800B11D242046BDE8CE
:105E7000F0810000ECB301002DE9FE4F06464D48CD
:105E8000894615460178012907D0EF224AA1002052
:105E9000FFF74BF80220BDE8FE8FC1784FF0010AF2
:105EA00019B9C660066180F803A080468078032790
:105EB000002869D1D8F8101042468E4201D1012045
:105EC00000E000202944C8F8101048B39068C0F1E1
:105ED0003004AC4200D92C46444A4946104422467C
:105EE000FAF7FEFAD8F808002D1B2044A1442644F6
:105EF000C8F80800302839D3444602D14FF00100D9
:105F000001E04FF0000040F211122BA1FFF70DF855
:105F1000D4E9021201233548FFF752FE607001E018
:105F200088F8017001A8009002AB0122444698F85D
:105F30000100D8F80C10FFF791FE08BBFFF76AF9D3
:105F400028B12A496078A268FFF77CFFC0B9A07821
:105F50004FF49A7280F0010017A1FEF7E6FF019856
:105F600000F02CF960B984F802A002E098F8020071
:105F700098B144461D49D4E9022000F083F808B1E5
:105F8000277088E7A07840B12A464946304600F09D
:105F900079F810B188F800707DE72A464946304606
:105FA000FFF7E6FE0028ECD0022188F8001013204D
:105FB00071E70000300000202E2E2F2E2E2F2E2EC7
:105FC0002F736F757263652F6461706C696E6B2FD0
:105FD000647261672D6E2D64726F702F666C6173D1
:105FE000685F6465636F6465722E6300A0060020BD
:105FF00010B5EFF3108472B6FBF7EEFA84F3108855
:1060000010BD0000FEB5184E054672787468AA42AD
:1060100026D0002772B194F83800800700D5F5B972
:106020000097019702976168002304F1180002F0BD
:1060300051FC38B19DB194F83800800704D57078D0
:1060400010B10CE00C20FEBDCDE90057029721688D
:10605000002304F11800F26802F03CFC10B17570E6
:106060000020FEBD0B20FEBD2801002001444FF49E
:106070000022491E904203D2914201D20120704772
:10608000002070472DE9F0473D4E0546002470780A
:1060900017468846012807D07B223AA10020FEF748
:1060A00044FF0220BDE8F087F0784FF0020A50B9B3
:1060B000284602F029FA040002D086F801A05CE02C
:1060C0000120F0707561B068B5FBF0F100FB115173
:1060D0006A1A7169B1FBF0F300FB1310081A8242CF
:1060E00004D0284600F026F90400E6D13069B5FB5B
:1060F000F0F100FB11516A1A7169B1FBF0F300FB7A
:106100001310081A824204D0284602F0FDF9040058
:10611000D3D1B1464E46D6E901010844A84207D87A
:10612000284600F007F9040002D089F801A024E015
:106130000FB3D6E903010844A84204D8284602F068
:10614000E3F90400F1D17068B168B146281A0E1A5B
:10615000B74200D23E461849324608444146FAF753
:10616000BFF936B1002089F802003544B044BF1BA6
:10617000D0E70120F7E7C9F81450204692E7000065
:10618000440000202E2E2F2E2E2F2E2E2F736F75B3
:106190007263652F6461706C696E6B2F64726167E6
:1061A0002D6E2D64726F702F666C6173685F6D6108
:1061B0006E616765722E6300D006002070B51F4DBA
:1061C0000446687808B1472226E024B3606810B31B
:1061D000A06800B3E068F0B12069E0B16069D0B1B7
:1061E000A069C0B1E069B0B1FF224FF480611448EA
:1061F000FAF72FFA0126AE700020E8706860A860F8
:10620000E8602861C5E9050420688047040008D1DA
:10621000287838B110E04D220AA10020FEF785FE53
:10622000022070BDA86900698047040004D0A869F5
:1062300040688047204670BD6E70FBE74400002038
:10624000D00600202E2E2F2E2E2F2E2E2F736F7560
:106250007263652F6461706C696E6B2F6472616725
:106260002D6E2D64726F702F666C6173685F6D6147
:106270006E616765722E630010B50446FFF7D8F8AB
:106280000148047010BD00004400002070B5154C9A
:106290000025607810B1012807D00AE0CC2212A1B5
:1062A0000020FEF742FE022070BD002000F042F800
:1062B0000546A069406880470646FF224FF480618A
:1062C0001648FAF7C6F90120A0700021E17061605C
:1062D000A160E1602161616161700EB1304670BD05
:1062E000284670BD440000202E2E2F2E2E2F2E2E3D
:1062F0002F736F757263652F6461706C696E6B2F9D
:10630000647261672D6E2D64726F702F666C61739D
:10631000685F6D616E616765722E6300D006002054
:1063200010B5EFF3108472B6FBF794FC84F3108879
:1063300010BD000070B50E4E05460024B07840B97F
:10634000B0690C498368D6E90102984704460120E8
:10635000B070FF220748B168FAF77BF9B068B5FB67
:10636000F0F100FB1150281A7060204670BD00004B
:1063700044000020D00600200748006948B10648C4
:106380000069D0F89C0120B103480069D0F89C0155
:1063900070470148001DFBE7ECB30100802807D0DF
:1063A00040B1054920F0800001EB0010103070472B
:1063B0000148FBE700487047005C0020074800697F
:1063C00048B106480069B0F8A00120B1034800694F
:1063D000B0F8A001704701484088FBE7ECB301002A
:1063E0000022034611461046184700000E4910B51A
:1063F00009690E4B0C3109E0824206D84A68824294
:1064000003D30868D860086910BD14310A68002AEF
:10641000F2D14C68002CEFD198680028F4D00168C4
:10642000D960006910BD0000ECB301002801002014
:10643000002070470348D0F81C0108B100207047C5
:106440000120704700301442474810B5016801230D
:1064500001B903600020454C014604EB8002C2F8FC
:106460004011401C0528F8DB4148016054F88C0FAE
:1064700020F0706040F0A06044F804093C48843883
:106480000360001F03603A4880380360206820F4EE
:10649000700040F480102060206820F4702040F4E8
:1064A00080302060206820F0706040F080702060B4
:1064B000206820F0704040F0005020602C487C386C
:1064C00003602B4890380360206820F4706040F42B
:1064D0001060206026488C380160206820F47040ED
:1064E00040F41040206022486C300360A06820F027
:1064F000F00040F05000A0601E48026822F0010247
:106500000260026842F002020260021F1160016034
:106510000521022004F0A6F80421022004F0A2F8CC
:106520000621022004F09EF81348016841F004019E
:1065300001600D485438016841F08071016000200D
:1065400003F0EEF8D4F8C00120F08000C4F8C001D8
:106550004FF0E0214FF40030C1F88001BFF34F8FBE
:10656000BFF36F8F10BD00005804004000A0004032
:1065700098191442040D00400008004070470000C4
:106580000349012802D00120086070470020FBE782
:10659000181914420349012802D0012008607047ED
:1065A0000020FBE7141914420349012802D00120FE
:1065B000086070470020FBE71019144210B50E4C1C
:1065C000E07978B9FFF734FF48B10C480068C0693A
:1065D000804700280FD103F0D3F801200AE0E079CA
:1065E000002808D0FFF724FF002804D1022003F080
:1065F000C7F80020E07110BD04010020B4B801000C
:106600002DE9F04385B081460D481D461646884663
:10661000DDE90C410DC802AF87E80D00B81C04F09D
:1066200042F80020CDE900478DF812002B46324693
:106630004146484602F014F905B0BDE8F083000079
:1066400068B50100092800D927303030C0B2704742
:106650001CB501AA69460A48FAF793FF002807D03B
:106660000198402805DD312206A10020FEF75DFCDF
:106670001CBD40220020009903F0E2FE1CBD00007A
:10668000646400202E2E2F2E2E2F2E2E2F736F752A
:106690007263652F7573622F6869642F7573626406
:1066A0005F757365725F6869642E630070B5164C20
:1066B00000204DF6FC756060A0602946E060FFF7A1
:1066C000D5FC20B129460020FEF716FF60600F4D73
:1066D0004FF4803629463046FFF7C8FC20B12946E2
:1066E0003046FEF709FFA0604FF400554FF4FC263A
:1066F00029463046FFF7BAFC002804D02946304628
:10670000FEF7FAFEE06070BDE4000020FCDF06004A
:1067100000487047F400002010B50C212020FFF73E
:10672000A5FC002809D00020054A016A914203D146
:10673000406A0449884201D0002010BD012010BDEC
:10674000939D939B0699969710B5FFF7E5FF002858
:1067500001D00020806A10BD0148406870470000E9
:10676000E40000200148806870470000E400002039
:1067700000487047C4360020004870478236002029
:10678000004870477536002000487047A336002047
:10679000004870474436002000487047CD3600203E
:1067A00000487047FE00002070B5FFF77FFF2048CB
:1067B00000F0D6FF01F022FE1D4831212030F9F70C
:1067C00072FF1B481B492030F9F77EFE1949184813
:1067D000491D2030F9F778FE15495E31A1F13E00E0
:1067E000F9F772FE1249A031A1F18000F9F76CFEB1
:1067F0000F4800242030F9F7FDFD0D4AC1B20220F8
:10680000A93200EB410010700320507002200023D9
:10681000A2F1890508E02E5D1654401CC0B2135445
:10682000401C641CC0B2E4B28C42F4D370BD0000C2
:1068300024360020F400002010B5124C207830B12E
:10684000622211A10020FEF770FB022010BD002281
:1068500011461046FAF7FEFE08B11E2010BD0020BA
:106860006070A070E070A060E060207120616061E5
:10687000A0614FF400511248F9F7F3FE0120207097
:10688000002010BD600000202E2E2F2E2E2F2E2E29
:106890002F736F757263652F6461706C696E6B2FF7
:1068A000647261672D6E2D64726F702F6961705F05
:1068B000666C6173685F696E74662E630000000029
:1068C000D00A002070B50E4D2868002816D100248B
:1068D000FFF774FD0B4A08E029B10988814202D113
:1068E00052F8240009E0641CE4B252F824104B1C56
:1068F000F2D12868002801D10348286070BD00004B
:106900006C040020700400203CBE010010B5002380
:1069100005E0DC0021FA04F4C4545B1CDBB29342B2
:10692000F7D310BD2DE9F0472E4F04468A4638783C
:1069300016464FF46041012808D040F279122AA18E
:106940000020FEF7F2FA0220BDE8F08788464445B1
:1069500001D32320F8E7FEF75DFE98B3C4F5604548
:10696000281FB04201D9324600E02A1F5146B869BB
:10697000FEF7EAFD4FF400590146B8614C4507D2D5
:106980002748324620445146F9F7AAFD0020DBE7AC
:10699000A019404523D10AEB050010F8023C30F85D
:1069A000042DC07863F31F4242EA0060814201D0A7
:1069B0002720C9E7524631462046FFF7B1FC10B107
:1069C0002020C1E70BE04A4615490020FEF7E8FD0C
:1069D0000446FFF76BFE012078702046B4E72620BE
:1069E000B2E70000600000202E2E2F2E2E2F2E2E1C
:1069F0002F736F757263652F6461706C696E6B2F96
:106A0000647261672D6E2D64726F702F6961705FA3
:106A1000666C6173685F696E74662E6300000000C7
:106A2000D00A002010B504460F484FF460410078AA
:106A3000012807D040F2BB120CA10020FEF775FA26
:106A4000022010BD8C4201D3232010BDFEF7E2FDD1
:106A500000B10CB1262010BD00202022BDE810405E
:106A6000D102FEF79DBD0000600000202E2E2F2ECB
:106A70002E2F2E2E2F736F757263652F6461706CCD
:106A8000696E6B2F647261672D6E2D64726F702F4B
:106A90006961705F666C6173685F696E74662E63AE
:106AA000000000000246084810B500EB810050F8D5
:106AB000040C002806D0114601F004FABDE810408D
:106AC00001F0F0B910BD00003C60002007494FF410
:106AD0008030086001F026FC00F0B2F90022114677
:106AE000034800F0F5F900F0B1F9FEE708ED00E029
:106AF000456B0100024901224A700871704700008D
:106B000004010020024901220A70C8707047000089
:106B100004010020024901228A7048717047000078
:106B20000401002002484FF40061006900F0AAB996
:106B30000401002002480421006900F0A3B900000C
:106B4000040100204FF00008474646461625FEF790
:106B500071FB00F0B7F9DFF85CB2CBF81000FFF77B
:106B600073FC4046FFF716FD3846FFF709FD304637
:106B7000FFF71AFDFAF7A0FC8F4C2088012800D0FF
:106B800000204FF495728DA1FEF7CFF9E06E00B1B1
:106B90008047FFF797FE9648006810B1C06800B1C3
:106BA0008047207B800702D5012002F08FF8207BF0
:106BB000C00702D00120FFF75FFBFFF7F5FDFEF7EE
:106BC000DBF903F0D1FCFEF7D7FB00285CD00020F6
:106BD00004F03CF8002003F0F3FB012100238BF8C4
:106BE00008104FF00B091A46824800F097F903216C
:106BF00000F09CF94FF0000A4FF0FF32002140F600
:106C00003F2000F051F984B2A00507D59BF806009B
:106C100010B1012000F006F9FCF7E8FD600702D58D
:106C2000022002F0ADFDE00613D5032002F0A8FD1E
:106C30000020FFF7A3FC002003F0C2FB0020FFF7B9
:106C4000A9FC0020FFF79CFC0020FFF7ADFCFEF73D
:106C500091F9A00602D5032002F092FD200501D58E
:106C6000FEF7BCF9200701D5FEF781F9E00741D016
:106C70005A2004F017F89BF8080006283AD2DFE8FB
:106C800000F02D0E2D1D39050120A1E78BF808A07D
:106C90000020FFF773FC002003F092FB2AE0B9F11B
:106CA000000F04D0A9F101005FEA000922D1012000
:106CB00003F086FB03218BF808101AE003F078FB41
:106CC00018B10120FFF75AFC0BE00DB16D1E11D178
:106CD0000120FFF753FC8BF808A00BE003F068FBE2
:106CE00018B102208BF8080004E08BF808A04FF0E0
:106CF0000B091625A0077FF57FAFFFF75FFCFEF7B6
:106D000035F99BF800005C4658B1E078012825D0A1
:106D1000022823D04FF0000884F800A04046FFF777
:106D200039FCA07850B16079012827D0022825D0FD
:106D3000002684F802A03046FFF736FC6078002871
:106D40003FF45AAF2079012826D0022824D000270A
:106D500084F801A03846FFF713FC4DE7B8F1010FA6
:106D600001D0012100E000215FEA0108D6D101280D
:106D7000D4D184F800A084F803A0CFE7012E01D07D
:106D8000012600E00026002ED5D10128D3D184F8B9
:106D900002A084F805A0CEE7012F01D0012700E072
:106DA0000027002FD6D10128D4D184F801A084F87F
:106DB00004A0CFE704010020ECB301002E2E2F2EFB
:106DC0002E2F2E2E2F736F757263652F6461706C7A
:106DD000696E6B2F696E746572666163652F6D6194
:106DE000696E5F696E746572666163652E6300002B
:106DF0006C040020D198010001498871704700009F
:106E000004010020FEF7E6BF10B5044640F2011170
:106E1000F9F727FC00F038FD00202070BDE8104095
:106E2000FEF7D8BF80B2DFF808C000DF002070474F
:106E3000397A0100DFF804C000DF704721820100C9
:106E4000014900200860704744040020002070477A
:106E500089B2DFF808C000DF00207047CD7D010057
:106E60000248DFF80CC000DF00487047F8630020DC
:106E70000D7D0100DFF808C000DF00207047000032
:106E80001D7D010010B50C460146EFF30380C006DE
:106E9000A0B202D0FFF706FE02E0DFF808C000DF74
:106EA000204610BD997A010091B280B20022DFF82D
:106EB0000CC000DFDFF808C000DF7047F97A01007E
:106EC000417A0100DFF804C000DF7047158301003C
:106ED00070B50D4C06460025206860B100231A46A7
:106EE0000B213046DFF824C000DF05462068401C37
:106EF0002060284670BDF9F783F9054A05493046F8
:106F0000DFF814C000DFF1E744040020998201009B
:106F1000506000200A20030091800100024A0146CF
:106F20000020516070470000440400200548002301
:106F3000054A816048F60B010448DFF814C000DF01
:106F40000020704744040020706300202D8201005F
:106F500099820100012805D0022805D003280BD012
:106F6000C72202E0BB2200E0BF2204A10020FDF7FF
:106F7000DCFFFBF7A7FCFEE7C322F6E72E2E2F2E41
:106F80002E2F2E2E2F736F757263652F72746F7391
:106F90002F5254585F436F6E6669672E630000007E
:106FA000FEE70000074801684FF0E0204161002142
:106FB0008161072101610448016841F07F4101605E
:106FC0004017704720BE010020ED00E07047704779
:106FD0002DE9FF5F8846DDE90FA5044600EB0806B2
:106FE0000020DDF838B0286092489146007930B131
:106FF00020783A2840F0BA808E49002008718D48E8
:107000008D4FC078C8B18B490020C8703A78391DBF
:107010000398F9F765FA38780399014403912968D0
:10702000084428608348C168B7F801006FF30F0176
:107030000843397801447F48C160B44218BF7D4F8E
:107040007ED020780A2818BF0D287AD03A282AD076
:107050003978002900F0DF8010F0100F00F00F00E9
:1070600008BF093000F00F0273487978435C1A4377
:107070004254491CC9B2797090F800E00EF1050045
:1070800081426DD300216C4B08461EF1050213D0DE
:1070900013F800C0401C6144C0B2C9B28242F7D8A4
:1070A00051B1042763E025216348F9F7DAFA00209B
:1070B00038707870B87055E0B87800284DD15E4BC4
:1070C0000120B870B3F8010040BAA3F80100D978E4
:1070D00004297DD005DC69B1012962D0022962D082
:1070E0003BE00A2902D00D2904D036E0988840BA46
:1070F000F88032E0F98839B1504A1288914203D0C1
:107100004F4A1288914248D1F9680A466FF30F023C
:107110001043884204D00120F8700227641C26E046
:107120000020F870724647490398F9F7D9F94248A8
:10713000017803980844039028680844286001E017
:1071400014E00FE03C49F868B1F801106FF30F004C
:107150000143394800780844F8603878002866D040
:1071600000203870641CB4427FF46BAF002728689D
:10717000FF22ABEB00010398F9F76BFA2D48296861
:10718000C068401ACAF80000301BA8EB0000C9F81C
:10719000000004B03846BDE8F09F01203871002798
:1071A000E5E70127E3E72868FF22ABEB000103983E
:1071B000F9F74FFA2868F968081ACAF80000301B76
:1071C000A8EB0000C9F800001B480179090300E0A2
:1071D00007E0407941EA0010F86004B00220BDE801
:1071E000F09F2868FF22ABEB00010398F9F731FA12
:1071F0002868F968081ACAF80000301BA8EB0000DC
:10720000C9F800000C48808840BA0004F86004B057
:107210000220BDE8F09F7978252908D210F0100FE0
:1072200000F00F0008BF09300001034A505401204C
:1072300097E700007C000020D02A00208600002074
:1072400084000020D42A00207FB50C4D0446284637
:10725000FEF7CEFE002810D1FF2210216846F9F774
:10726000F8F920680090606801902089ADF8080066
:107270006A4610212846FFF753F87FBD00E007005B
:107280002DE9F05FDFF8F8800446154698F8000015
:107290008B464FF4604A012805D0A22239A1002074
:1072A000FDF743FE3EE02020B4FBF0F3020200FBBA
:1072B0001343114602260BB1AB222DE0202D04D33F
:1072C000B5FBF0F300FB135008B1B22224E0B4FB8D
:1072D000F1F002FB10402844884201D9B9221BE09A
:1072E00098F8020078B998F8030050B1D8F808006F
:1072F000844204D3D8F80C100844A04203D8C72213
:107300000AE0C12208E098F8040070B1D8E904014D
:107310000844A04209D0CF221AA10020FDF705FEA3
:1073200088F800600220BDE8F09F6719B4F5FC2FD3
:1073300002D2B7F5803F17D84FF0010988F80490C2
:107340002A4659462046C8E90445FFF7EBFA2628A5
:1073500004D00028E7D088F80060E4E75A462946C0
:107360002046FEF7DDFF18B188F800602020DAE73C
:10737000574503D3FFF79AF988F801900020D2E728
:10738000600000202E2E2F2E2E2F2E2E2F736F7585
:107390007263652F6461706C696E6B2F64726167D4
:1073A0002D6E2D64726F702F6961705F666C6173F2
:1073B000685F696E74662E630000000020207047CD
:1073C00070B514460E46054620444FF48061B1EB7B
:1073D000402F07D240F263220AA10020FDF7A5FD4D
:1073E000002070BD4FF400713046F9F73AF935B915
:1073F00011481249006942013046F9F771F86002FC
:1074000070BD00002E2E2F2E2E2F2E2E2F736F7557
:107410007263652F6461706C696E6B2F6472616753
:107420002D6E2D64726F702F7669727475616C5F4A
:1074300066732E6300000000A400002024320020A8
:1074400010B50B464FF4007408B1002010BD224661
:1074500002491846F9F744F8204610BD642F002071
:107460002DE9F04F8A46410287B000234FEA422BB4
:107470001D460693029130B1BAF1000F03D00020EF
:1074800007B0BDE8F08F344C2078012841D00228A5
:1074900041D0002631A0009059465046029A03F090
:1074A0004DF90746304931A0CDE900013B46594628
:1074B0005046029A01F0D4F9074461882DA0CDE925
:1074C00000013B4659465046029A02F00DFDC41990
:1074D0004EB12AA0CDE90006234659465046029AED
:1074E00001F0BEF9044406A8FDF74CFF060030D0B9
:1074F000069870B323A00090234659465046029A3E
:1075000003F01CF9044403AF4FF00A084FF400796C
:1075100019E01FA6BEE721A6BCE723A003AB07C85E
:1075200083E80700069850F825106D1CEDB203A8FB
:1075300003F0B9F8CDE90078234659465046029A3F
:1075400003F0D8F80444B54203D204F10A004845D8
:10755000E3D3204694E700009C000020417373654C
:1075600072740D0A00000000202D002046696C6531
:10757000000000004C696E6500000000536F7572DA
:107580006365000048657864756D70730D0A0000CE
:10759000426F6F746C6F6164657200004170706C53
:1075A00069636174696F6E000000000000000000F4
:1075B0000D0A000030B413460C464202204630BC8F
:1075C000590202F0E5BC00002DE9FE4F04464002DE
:1075D0008A464FEA422B0026029003F05BFB0546E9
:1075E000FEF7DAF807462846FEF7FAF805462CB10A
:1075F000BAF1000F02D00020BDE8FE8F20A0CDE937
:107600000007334659465046029A01F029F90446CC
:107610001DA00090234659465046029A03F08EF86A
:107620000026044401274FF00208DFF8649019E0B7
:107630004FB918A1CDE90018234659465046029A81
:1076400003F058F80444E8070AD059F826000090DF
:10765000234659465046029A03F070F80444002726
:107660006D08761C0DB1052EE2D30BA1CDE90018F3
:10767000234659465046029A03F03CF82044BBE7A3
:107680006572726F72000000747970653A200000B4
:1076900054B501002C2000000D0A0000F8B5460288
:1076A00055020F46002310B10FB10020F8BD0D4860
:1076B000009032462946384603F040F804460AA0B6
:1076C00000902346324629463846FEF72DF90444F9
:1076D00006A00090234632462946384603F02EF88D
:1076E0002044F8BD00C201004052000022293B0D99
:1076F0000A3C2F7363726970743E0D0A3C2F626FEF
:1077000064793E0D0A3C2F68746D6C3E0D0A0000D2
:107710002DE9F041094C06460D462046F8F76AFE71
:10772000074645B116B10020BDE8F081024621466A
:107730002846F8F7D5FE3846F6E7000028C10100D4
:1077400010B50B464FF4007408B1002010BD22465E
:1077500002491846F8F7C4FE204610BD642D0020EB
:107760000449D1E900235A40D1E902314B405A4043
:10777000026070471810004010B5084654022146B8
:10778000F8F76FFF204610BD70B5244D4FF0FF3461
:107790006878A978884201D0012000E0002040F2FA
:1077A000F9121FA1FDF7C1FB6878022803D0C0B110
:1077B00001281AD022E027484FF4FA7490F82000EC
:1077C000E0B101280AD0022818D0032816D040F2D0
:1077D0000B2213A10020FDF7A8FB0FE044F6206464
:1077E0000CE0A878022808D008E0A878022801D088
:1077F00018B103E040F6C41400E00024601C05D179
:1078000040F21B2206A1FDF790FB0024A868A042CD
:1078100001D9012070BD002070BD00008C00002047
:107820002E2E2F2E2E2F2E2E2F736F757263652FF7
:107830006461706C696E6B2F647261672D6E2D646C
:10784000726F702F7666735F6D616E616765722E01
:1078500063000000F82C002070B5202903D000231D
:107860001A4601260CE090FAA0F070BDC40704D0BF
:107870008D1A6D1E06FA05F423434008521CD2B23D
:107880008A42F3D3184670BD10B525210648F8F793
:10789000E8FE06480021C160017041708170C1702E
:1078A000C180017110BD0000D02A00207C000020A2
:1078B0000D4810B5002101604160816020210B4816
:1078C000F8F7CFFE0A49D1F8800240F05300C1F822
:1078D00080020120402201EB8003C3F88022401C7B
:1078E0000828F8D310BD000034040020905E00206A
:1078F0000000104070B505460E460846F8F77AFDC0
:10790000401C3C2801D93C2003E03046F8F772FDCA
:10791000401C0446024631462846F8F7E1FD0020A7
:1079200085F83B00E0B270BD0146EFF3108000F037
:10793000010272B6086808B103680B60002A00D122
:1079400062B6704770B50D46002812D04FF6FF7131
:10795000084C884204D222680146104600F0D4FA4E
:1079600020684570044800F0F8F8BDE8704000F069
:1079700087BB70BD580400200464002070470000DD
:1079800070B51A4EF06800282ED0B08A401EB08222
:10799000002523E0A06838B161684160606810B1DB
:1079A000A16881606560A56010482146183800F024
:1079B000CFFAA08AB0826078042804D10C49E08A0A
:1079C00009880844A0820120607084F82000E068E3
:1079D000F060E06808B10661E5602561B08A0028C2
:1079E00002D1F468002CD5D170BD00001C640020C9
:1079F0006004002070B504000FD00D4DA178012661
:107A00002868827891420CD900F0BEFA2868467046
:107A10002046BDE8704000F033BB064800F09DF8FA
:107A2000F7E766702146BDE87040024800F090BA62
:107A300058040020046400200321FFF783BF0000E6
:107A400001480068408B70475804002010B5044678
:107A5000008B084320836278618B062A16D0052AA2
:107A600017D1084215D001EA0002628388432083BF
:107A7000204600F0ADFA01206070022084F820005A
:107A80002146BDE81040034800F062BA31EA000226
:107A9000ECD010BD04640020024670B5154800EB20
:107AA000810050F8044C002C22D0208B10432083FE
:107AB0006178658B062918D0052919D1284217D07D
:107AC00005EA00016183A8432083204600F080FA84
:107AD000208BA843208301206070022084F82000BE
:107AE0002046BDE87040FFF785BF35EA0001EAD0C7
:107AF00070BD00003C60002070B503460C480D4688
:107B00000468208B42B133EA000101D0062109E06C
:107B100098432083022070BD10EA030101D06183E5
:107B2000F6E7052163832846FFF70CFF012070BDAF
:107B300058040020814202D342688A4201D80120C1
:107B40007047EFF3108212F0010F72B603680B60FA
:107B5000016000D162B600207047014640680023F2
:107B600042684A600A78022A05D0012A03D0032A13
:107B700001D04360704742680AB1916043608360FE
:107B80007047000070B504460020154620700122A1
:107B90006270A1706060A060E0602061A082E082FD
:107BA0002083608384F8200084F82100608C18B959
:107BB0000448FFF7B9FEA06229462046BDE87040A0
:107BC00000F004B8805F00207047000010B5428CC0
:107BD000920803D10E4A1288C2F38D02836A03EB26
:107BE00082035A0700D51B1F4FF0807243E902122F
:107BF00000221446403B43F82240521C0E2AFAD37E
:107C0000C2691A624362C162806A0249016010BDA2
:107C10001CBE0100A52E5AE20349044A0968C88225
:107C200012881044888270475804002060040020A5
:107C30000748016807488A8A0088CB8A101A1A44C4
:107C400080B28A82010402D40421FFF77BBE704710
:107C500058040020600400202DE9F04104464068EB
:107C60000F46002620B16078022818D0A08980B382
:107C7000A089E189884241D2208904EB8000076114
:107C800072B6A089401CA08162B62089401C80B2D7
:107C90002081E189884200D12681BDE8F0816670AB
:107CA0002046FFF75AFF80F820602189054604EB43
:107CB0008101C069086172B6A089401CA08162B6CA
:107CC0002089401C80B22081E18988420BD1268125
:107CD00009E0FFE72046FFF740FF0546C0690421A1
:107CE000076085F8201001206870284600F070F9C0
:107CF0002946BDE8F041044800F02AB9BDE8F0414A
:107D00000320FFF727B9000004640020032101705D
:107D10000021417041804160816070472DE9F0474A
:107D20000446408820B1274EA1683268914202D0B3
:107D3000FF20BDE8F087401E0004000C60803ED1AB
:107D400031686078DFF88080887061684FF00009E2
:107D5000012739B32046FFF700FF0546052085F8C7
:107D60002000284600F034F96780A560A87860708C
:107D70003168D8F804008A788078824201D3284696
:107D80000AE0114800F0E4F829460F4800F0E0F856
:107D9000306847706F7010E0FFF72CFE316881F893
:107DA00020900CE0D8F804108A783168824206D915
:107DB000054800F0CDF8306847700020ECE700205F
:107DC000B7E70000580400200464002070B5184D87
:107DD0000E4604464188286839B1A168814208D11D
:107DE0006088401C6080002070BDA060807860705A
:107DF000F6E776B162788078824203D28870A06814
:107E000000F0CCF8606830B12046296800F0A0F896
:107E100008E0012070BD2868606029680020486083
:107E20002868846009213046FFF78CFDF1E70000E7
:107E30005804002070B5184801210268517000688C
:107E400000F0A2F8154D6C7812E005EBC40148680B
:107E50000278C2B1012A1BD000F0E6F8E878641C71
:107E6000844200D1002472B6A878401EA87062B681
:107E7000A8780028E9D16C700948FFF76EFEBDE8CC
:107E8000704000F0FDB8098989B2FFF7DFFDE5E732
:107E90008968FFF7E1FEE1E7580400201860002040
:107EA000046400200548017811B101214170704738
:107EB00003494FF0805008607047000050040020D4
:107EC00004ED00E0F0B40F4FBC1CFE783D4672B6E6
:107ED000BA78B24207D2521C22702A78531CB3429D
:107EE00000D100232B7062B6FB78934205D907EBD3
:107EF000C202C2E90101F0BC7047F0BC0220FFF7EA
:107F000029B8000018600020104A10B5D368ABB142
:107F100013469B8A03E08CB12246A48A2344D4688A
:107F20008B42F8D3C460D0600261C46804B12061A0
:107F3000591A8182908A401A908210BD0024C46030
:107F4000D060C91A02619182848210BD1C64002035
:107F500030B502780024022A03D0012A01D0032A76
:107F600000D101248B7800E01046426812B1957868
:107F70009D42F9D24A6041601CB102B191608860B3
:107F800030BD0020FBE7000003494A684260002240
:107F900082604860704700000464002010B5836868
:107FA00004462BB9607801280ED1084B03E09B688A
:107FB00018780028FBD0204600F01EF82146BDE8C6
:107FC00010401846FFF7C4BF10BD00000464002035
:107FD00010B5016900290ED0C268CA60C3680022CA
:107FE0003BB18B8A848A23448B82C3681961C26047
:107FF00000E08A82026110BD816839B142684A603E
:108000004168002901D0806888607047054906E012
:108010004A68824202D14068486070471146002990
:10802000F6D170470464002010B5416879B1FFF7BC
:1080300094FD0446FFF7CCFF01206070032084F814
:1080400020002146BDE810400348FFF781BF41886A
:10805000491C418010BD00000464002006480068EF
:10806000D0E90910814203D300680449884202D054
:108070000120FEF76FBF704758040020A52E5AE27A
:1080800002494860022141707047000058040020F6
:108090002DE9F0471646414A8146884600200546AC
:1080A0003D49128802E041F82050401C9042FAD32A
:1080B0003B48302201883B48FCF7F4FE3A480088F0
:1080C00080B240F00042394801683948FCF7EAFEC6
:1080D00038480822018838480068FCF7E3FE374C2E
:1080E000FF27374AE770658400212046FFF74AFDE5
:1080F000344804210170456033480170C560056152
:108100008582606A2030F8F775F83048314904609C
:10811000022060702E48057045700978C170FFF725
:1081200053FD2D48016841F47F0101600068390664
:1081300001EA00202849C0431439B0FA80F00968E8
:10814000C0F10800C1F30221814200DB481C224932
:10815000091F0B686FF08072824063F317020A6098
:10816000FEF720FF1D49002808600DDB00F1E0212B
:1081700081F8007400F01F0201219140401180003D
:1081800000F1E020C0F80011324641464846BDE803
:10819000F047002300F080B83C6000201ABE0100C8
:1081A00030BE0100B05E00201CBE010034BE0100E4
:1081B000805F00203ABE01004004002034640020AB
:1081C000A16F0100046400201C64002058040020FA
:1081D0001860002038BE010020ED00E054040020AB
:1081E0000C4810B50268012151700068FFF7CCFE01
:1081F000FFF7C4FB08480168491C0160FFF7C0FB9A
:1082000000F02AF80548FFF7A8FCBDE81040FFF78A
:1082100037BF0000580400206004002004640020E0
:10822000014800687047000060040020074CDFF838
:1082300020C0208980B200DFDFF818C000DF61684D
:108240000029F9D000208847F6E700004404002008
:10825000197C0100317C010070B50D4D28680028A3
:1082600015D0A8880B4E401EA8800AE0E088FEF7D3
:10827000AEFEA088A8802068286021463068FFF7FD
:1082800059FCA888002802D12C68002CEED170BDC2
:1082900064040020400400202DE9F0411E461746EA
:1082A00080460C4611F0FF0F00D14C1C1548FFF71B
:1082B0003BFB051E23D0200AAF626884E1B2424630
:1082C0002846EE61FFF75EFC104901240E4809883C
:1082D00005E000EB840252F8042C1AB1641C8C42B5
:1082E000F7D9002400EB840040F8045CEC702846C9
:1082F000FFF780FB0648006880F820402046BDE874
:10830000F0810000B05E00203C6000201ABE010039
:108310005804002002480068002800D0C078704748
:108320005804002070470000F0B5294A00214FF49E
:108330007F64136823FA01F2B2FBF4F2491C904205
:1083400001D20929F6D3904241D3224A14688C42C3
:1083500000D01160491ECB408100B3FBF1F1022235
:108360000904090C4FF0100531D009E0002A2ED085
:10837000521E92B225FA02F14143B3FBF1F189B2E8
:10838000FF29F3D801D011B102E0FE2100E0012164
:10839000D54005FB01F4B3FBF4F44E1C7543B3FB6D
:1083A000F5F3A04201D9041B00E0241A984201D938
:1083B000C51A00E01D1A084FAC427B6803D262F375
:1083C0001F21596002E062F31F265E60F860F0BD75
:1083D0002003002060040040240300207CB5DDE978
:1083E00006540CB103A400E003A4CDE9005400F04E
:1083F00037FA7CBD31000000300000002DE9F04765
:1084000000242646FDF7DAFFDFF8F4900546A04683
:108410004F4621213B48C9F81080F8F722F9394826
:1084200021212130F8F71DF9364809214230F8F7AB
:108430003AF987F81480334FA7F15E0AB8195AF851
:10844000241002F030F9641C3044E4B2C6B2042CAB
:10845000F4D307F8068000242A4F26462137A7F1D7
:108460006F0A38195AF8261002F01DF9761C2044BC
:10847000F6B2C4B2042EF4D307F80480214C464669
:10848000423420464F46D9F8001002F00CF9C0B231
:108490002654FDF771FF00683861194810300671E5
:1084A000280BFEF7CFF8164C15342070C5F30320C7
:1084B000FEF7C8F86070FCF75FFF01281AD0FDF7DF
:1084C0003DFBB8B1C5F30310FEF7BCF8A07005F092
:1084D0000F00FEF7B7F8E070094826711A30302116
:1084E000017032214170352181703821C1700671CF
:1084F000BDE8F087082040EA151000F00F00E3E720
:10850000E4000020823600202DE9F041364E074677
:10851000B0694169384688470546B069816938467F
:108520008847044635B12CB14FF4806845450AD8D8
:10853000012009E040F235122CA10020FCF7F5FCE7
:108540000220BDE8F08100204FF49D7227A1FCF7C6
:10855000ECFCB8FBF5F105FB118048B1002040F2BE
:108560003B1222A1FCF7E1FCAC4203D3012002E064
:108570000120F4E700204FF49E721CA1FCF7D5FC0B
:10858000B4FBF5F005FB1040C0B1002040F23D12F5
:1085900016A1FCF7CAFCB7FBF4F004FB1070381A04
:1085A000C6E903047060444500D34446B460B16931
:1085B000096A29B1884704000AD101E00120E5E7F2
:1085C000307850B1B069C168F0688847040004D0C1
:1085D000B069406880472046B3E7FF221048B16881
:1085E000F8F737F80020ACE7440000202E2E2F2E9D
:1085F0002E2F2E2E2F736F757263652F6461706C32
:10860000696E6B2F647261672D6E2D64726F702FAF
:10861000666C6173685F6D616E616765722E630081
:10862000D006002010B5094C207840B100F08AF83F
:108630006068C168064888470021217010BDC022CB
:1086400004A10020FCF771FC022010BD04000020F2
:108650009C0500202E2E2F2E2E2F2E2E2F736F7561
:108660007263652F6461706C696E6B2F64726167F1
:108670002D6E2D64726F702F66696C655F737472F6
:1086800065616D2E6300000070B5134C05462078BF
:1086900008B1852202E0022D06D38B220FA1002013
:1086A000FCF743FC022070BDFEF70CFCA0604FF409
:1086B00082711748F7F7F7FF0120207006480C3049
:1086C00000EB051060604168114888470028EAD037
:1086D0000321217070BD0000040000202E2E2F2EDB
:1086E0002E2F2E2E2F736F757263652F6461706C41
:1086F000696E6B2F647261672D6E2D64726F702FBF
:1087000066696C655F73747265616D2E630000004D
:108710009C0500202DE9F041094D0E460746002436
:1087200005EB0410314602683846904710B12046E8
:10873000BDE8F081641CE4B2022CF1D30320F7E71A
:108740001000002010B5FEF7BDFB0649896888427D
:1087500001D1012000E00020BDE81040622202A10A
:10876000FCF7E3BB040000202E2E2F2E2E2F2E2EE2
:108770002F736F757263652F6461706C696E6B2FF8
:10878000647261672D6E2D64726F702F66696C65FF
:108790005F73747265616D2E6300000010B500F1A7
:1087A000080103220C4607A0F7F743FE002806D075
:1087B0000322214604A0F7F73CFE08B1032010BDB8
:1087C000012010BD42494E004845580070B5154D76
:1087D00006460C462878012806D0A42212A10020C3
:1087E000FCF7A3FB022070BDFFF7ACFF68682246D0
:1087F00031468368194898470446132806D0142C3C
:1088000006D02CB103202870204670BD0220FAE764
:108810002878012800D00020B22203A1FCF785FBB4
:10882000F2E70000040000202E2E2F2E2E2F2E2ED9
:108830002F736F757263652F6461706C696E6B2F37
:10884000647261672D6E2D64726F702F66696C653E
:108850005F73747265616D2E630000009C050020DB
:108860002DE9FC478246DDE90A0700901C46904648
:108870008946504601F062FF054602260EA0CDE96A
:108880000006631942464946504601F033FF05444D
:108890006319424649465046009701F04FFF054490
:1088A00006A0CDE90006631942464946504601F04C
:1088B00021FF2844BDE8FC873A2000000D0A000093
:1088C00010B51E21002000F0C3FC002800D00120BC
:1088D00010BD00002DE9F04792B00D46DDE91A9871
:1088E00004461E46174644216846DDF870A0F7F797
:1088F000DAFECDE90076CDE9029860680990A068BB
:108900000D902068CDE90E054FF0807010906846FC
:1089100000F054FC00281DD0144DDFF854800024D2
:1089200011A9404600F0AEF998B11198800314D512
:108930006946002000F0F4F800280BD00D494046AD
:1089400000F0DAFC002805D00098BAF1010F08D039
:1089500050B1002012B0BDE8F087641CAC42DFD3F8
:10896000F7E7B9198842F4D10120F3E740420F003C
:10897000F0ED00E003005FA010B5044600F0C6FE75
:10898000002801D104F07F4010BD10B5F8F794FD28
:10899000F9F758F8012010BD2DE9F8430020411ED9
:1089A000009032486426042701600024DFF8C0806C
:1089B000416011E084B10121002000F049FC012058
:1089C00000F090F90220FEF72DFA002000F08AF95D
:1089D0000220FEF727FA0024FFF7D7FFD8F800009F
:1089E00010B1806800B18047F8F748FEA0B3FFF7E8
:1089F00067FF88B30021082000F02AFC60B34FF025
:108A0000A041042000F024FC30B300254FF02049A1
:108A100009E06946042000F0DDF8F0B1009939EA78
:108A2000010002D06D1CB542F3DBB54217D0012C1A
:108A300015D01049042000F00BFC68B1D8F80000F4
:108A400010B1006900B180470021082000F000FC4F
:108A500010B10120BDE8F88301E00124E5E77F1EA5
:108A600001247FB2002FA5DC0020F3E720010020C5
:108A70006C040020000F005010B5F8F78BFE0120A9
:108A800010BD0000F8B50D46044662B396081749BC
:108A9000002000F0DBFA002826D00527042221461A
:108AA0006846FDF733FF6946384600F0BFFA0128F3
:108AB00019D10F270021384600F0B8FA012812D149
:108AC0000024761E07E02946384600F0AFFA012858
:108AD00009D1641C2D1DB442F5D30E20294600F0A7
:108AE000A5FA012800D00020F8BD000052000023A4
:108AF00038B50D4604460949002000F0A7FA0028C1
:108B00000BD06946204600F035F8002805D0A007B4
:108B1000C10E0098C8402870012038BD50000023C5
:108B20002DE9F0410E46014600246425104800F06E
:108B3000E3FB002810D00E4F3F1F3146384600F0AF
:108B4000A1F8002808D03068C00302D4641CAC42ED
:108B5000F3DBAC4202D10020BDE8F081044831468D
:108B6000001D00F08FF80028F6D00120F4E7000087
:108B7000F4ED00E01CB50C460146042201A8FDF707
:108B8000C5FE052001A900F051FA012820D10F20CF
:108B9000694600F04BFA01281AD10E20694600F010
:108BA00045FA002222609DF8031042EA016121602B
:108BB0009DF8022041EA024121609DF8012041EA2E
:108BC000022121609DF8002011432160012800D07E
:108BD00000201CBD38B50C4600F00C006946801C16
:108BE00000F024FA002222609DF8031042EA01619D
:108BF00021609DF8022041EA024121609DF8012098
:108C000041EA022121609DF80020114321600128E2
:108C100000D0002038BD2DE9F04114460F4605462E
:108C200008E039462846FFF763FF002827D0641E76
:108C30006D1C7F1C14B3A807F3D111E0C5F3090024
:108C4000C0F58066B44201D224F0030632463946AC
:108C50002846FFF717FF002811D035443744A41BDE
:108C6000032CEBD808E039462846FFF741FF0028DF
:108C700005D0641E6D1C7F1C002CF4D10120BDE8C2
:108C8000F081000070B50C4605460749002000F051
:108C9000DDF9002806D021462846FFF76BFF0028A3
:108CA00000D0012070BD0000520000231CB5002040
:108CB0006A46FF211154401CC0B20828FAD311465D
:108CC0003320F9F7E9FC01201CBD000001490870C0
:108CD00070470000180100200149486070470000FB
:108CE000180100200649096811B1C96901B1084796
:108CF0000449096808B1002000E0012008607047BD
:108D00006C04002004030020F8B50224064606285F
:108D100001D0FFF73AFE4E494E4D4F1C082E74D23B
:108D2000DFE806F00415085A5C748A910120FFF709
:108D3000D9FF88E00120FFF7D5FF0220FEF772F887
:108D40000020FFF7CFFF0220FEF76CF879E0FFF775
:108D500023FE002878D0404E307801280BD00FE059
:108D6000641E64B2002C70DD0120FFF7BBFF0220FF
:108D7000FEF758F80020FFF7B5FF0220FEF752F883
:108D80003946284600F0B8FA0028E9D0314C0121D4
:108D90000C34204600F0B0FA002855D0307828B9BD
:108DA0000120FFF79FFF0220FEF73CF80020FFF7AD
:108DB00099FF0220FEF736F869462846FFF762FF62
:108DC000002841D000988003F6D50021204600F00D
:108DD00093FA002838D036E02846F8E7F8F74EFC3A
:108DE000002831D0FFF76CFD00282DD0002108208D
:108DF00000F02EFA002827D04FF0A041042000F008
:108E000027FA002820D03946E6E71EE0FFF7C4FD28
:108E1000002819D00E492846C91C00F06DFA002818
:108E200012D069462846FFF72DFF00280CD0009885
:108E30008003F6D507E007E0284600F05DFA002839
:108E400002D0F8F7A7FC0120F8BD0020F8BD000013
:108E500000005FA0F0ED00E018010020F8B502244A
:108E60000546062801D0FFF790FD6C492A46CE1C26
:108E70006B4D082A7ED2DFE802F00442089A9CB4C7
:108E8000C9C70120FFF72EFFBEE00120FFF72AFF30
:108E90000220FDF7C7FF0020FFF724FF0220FDF7A7
:108EA000C1FFFFF779FD00287ED069460420FFF757
:108EB00091FE002878D0009820F08041042000F036
:108EC000C7F9002870D069460420FFF783FE002808
:108ED0006AD000980028F6DB20F08051042000F0D2
:108EE000B7F9002860D069460420FFF773FE002818
:108EF0005AD000988000F6D4F8F74CFC84E0FFF7D5
:108F00004BFD002850D00FE0641E64B2002C31DD10
:108F10000120FFF7E7FE0220FDF784FF0020FFF7A6
:108F2000E1FE0220FDF77EFF3146284600F0E4F91D
:108F30000028E9D069462846FFF7A4FE002864D03F
:108F400000988003F6D5364C01210C34204600F001
:108F5000D3F9002859D0324E6946E43E3046FFF737
:108F600091FE002851D0009800F4E0612D4840683F
:108F7000014300E050E02C480143304600F0BCF9CA
:108F8000002842D00220FDF74DFF69462846FFF732
:108F900079FE002839D000988003F6D500212046BC
:108FA00000F0AAF9002800E02FE02ED02CE028469F
:108FB000F6E7F8F763FB002827D0FFF781FC0028CD
:108FC00023D00021082000F043F900281DD04FF0E5
:108FD000A041042000F03CF9002816D00F49491C9C
:108FE000E5E7FFF7D9FC00280FD03146284600F00E
:108FF00083F9002809D069462846FFF743FE002878
:1090000003D000988003F6D50120F8BD284600F073
:1090100073F90028F9D06FE70020F8BD00005FA0C9
:10902000F0ED00E0180100200000FA0570B50D46D3
:109030000646002429463046F8F7CAFE022803D126
:10904000641CE4B2642CF5D370BD000038B50D4645
:109050000446FFF791FC04F0F00240EA0201082008
:1090600000F0F6F8002805D034B90E484168A9424E
:1090700001D1012038BD456004F00C0404222946CA
:109080006846641CFDF742FC69462046FFF7CEFFA8
:10909000012805D10E200021FFF7C8FF0128E9D0E3
:1090A000002038BD20010020F8B50D4604462AB343
:1090B000960813490020FFF7C9FF00281FD0052795
:1090C000042221466846FDF721FC69463846FFF731
:1090D000ADFF012812D10D27002407E029463846AC
:1090E000FFF7A4FF012809D1641C2D1DB442F5D35C
:1090F0000E200021FFF79AFF012800D00020F8BDC4
:109100005200002370B50C46054608490020FFF7C1
:109110009DFF002809D0A807C00E04FA00F12846D8
:1091200000F02CF8002800D0012070BD5000002372
:1091300073B50646002464250F48019900F0DCF859
:10914000002813D00C4846F48031001F00F0D4F8FA
:1091500000280BD0084E083E01A93046FFF792FDCB
:10916000002803D00198C00301D501207CBD641CF8
:10917000AC42F1DB00207CBDF8ED00E038B50C46D8
:10918000014604226846FDF7C1FB05206946FFF74A
:109190004DFF012810D1042221466846FDF7B6FB99
:1091A0000D206946FFF742FF012805D10E2000215E
:1091B000FFF73CFF012800D0002038BD38B5054638
:1091C0000021082000F044F800283AD0002420466E
:1091D00055F82410FFF7ACFF002832D0641C042C93
:1091E000F5D30920696AFFF7A3FF002829D00D24D1
:1091F000204655F82410FFF79BFF002821D0641C5F
:10920000102CF5D31020296CFFF792FF002818D0FE
:109210000E4C0D49204600F06FF8002811D00A4985
:109220002046891E00F068F800280AD0694604200C
:10923000FFF7D0FC002804D0009810F0A00F01D058
:10924000002038BD012038BD0B005FA0F0ED00E02C
:10925000F8B50D4E04460D46082802D13068A842E4
:1092600010D004F00C0704226846FDF74FFB694656
:109270003846FFF7DBFE012801D00020F8BD082C9E
:1092800000D135600120F8BD200100202DE9F0411A
:1092900014460D46064608E029783046FFF732FFAF
:1092A000002827D0641E6D1C761C14B3B007F3D1C0
:1092B00011E0C6F30900C0F58067BC4201D224F07A
:1092C00003073A4629463046FFF7EEFE002811D044
:1092D0003E443D44E41B032CEBD808E0297830469B
:1092E000FFF710FF002805D0641E6D1C761C002CB3
:1092F000F4D10120BDE8F08170B50C460546074960
:109300000020FFF7A3FE002806D021462846FFF7DD
:1093100035FF002800D0012070BD0000520000235E
:1093200010B5FDF7CFFD07494968884201D10120FA
:1093300000E00020BDE8104040F2691202A1FBF7F6
:10934000F4BD00008C0000202E2E2F2E2E2F2E2E4E
:109350002F736F757263652F6461706C696E6B2F0C
:10936000647261672D6E2D64726F702F7666735F05
:109370006D616E616765722E630000000248002116
:10938000C068FDF765BD00008C0000200148C06882
:10939000FDF770BD8C00002002480078012800D045
:1093A000002070476000002002480078012800D0AB
:1093B0000020704728010020FEB51C4E34697CB3A4
:1093C00000250C341DE0FDF711F818B190F83800B5
:1093D000400715D4206800F059F900281FD101205A
:1093E000FCF710FE05001AD1009001900290104881
:1093F00000231A46406881681830FFF76BFA80B185
:10940000143420680028DED161680029DBD130697E
:1094100090F8A20110B100F075F805462846FEBD8F
:1094200001E01020FBE70120F9E70000ECB30100A8
:10943000280100203EB505461348006908B31348CB
:10944000446844B1284600F023F8B5FBF0F100FB76
:109450001150A0B901E002203EBD0120FCF7D2FD71
:109460000028F9D10090019002900346E1682A4655
:1094700004F11800FFF72EFA08B100203EBD0F20BE
:109480003EBD01203EBD0000ECB3010028010020DC
:109490000E4910B50A69BAB1916879B1491E0DD467
:1094A000526802EBC1031B68834205D8042000EB1D
:1094B000C1001044006810BD491EF2D54FF4C672B9
:1094C00003A10020FBF731FD002010BDECB301002B
:1094D0002E2E2F2E2E2F2E2E2F736F757263652F2B
:1094E0006461706C696E6B2F696E7465726661631E
:1094F000652F7461726765745F666C6173682E6353
:109500000000000070B5114D2869E0B1104C00203A
:1095100060706060012000F033F910B128690C30F0
:1095200007E0072070BD017AC90701D0A06006E0FE
:10953000143001680029F6D141680029F3D10120D7
:109540002070002070BD012070BD0000ECB3010050
:10955000280100202DE9FF5F81463E4816468846D7
:109560000069002874D03C48456885B13B480068D4
:1095700028B143691BB14846984701280BD0022007
:10958000FCF740FD4FF0000A002801D13BE002202B
:1095900004B0BDE8F09F0D20FAE76C6BB44200D92F
:1095A0003446686A22464146FFF770FE78B3686A1F
:1095B000CDE9000ACDF808A005F118005746296941
:1095C00023464A468346FFF785F908B3FBF71AFEA0
:1095D000B0B1686988B30320FCF714FD0028D7D127
:1095E00095F83800C00700D00120696ACDE900175E
:1095F0000290696923464A465846FFF76BF9D0B195
:10960000A144A044361B002EC7D10020C0E716E0BD
:109610001120BDE7102C01D2274600E010273A4662
:1096200069464846FFF7F7FA48B13A466946404668
:10963000F6F7B4FE28B11220AAE706E008E00A20F7
:10964000A6E7F61BB944B844E41B002CDBD0E1E7E5
:1096500001209DE7ECB30100280100206C040020EC
:1096600070B505460848006900280BD04FF4807497
:109670002846FFF70DFFA04203D22846FFF708FF58
:109680000446204670BD0000ECB3010070B5FCF745
:10969000ADFE040011D00B4D6868A0420BD0002035
:1096A000FCF7B0FC002807D1E26A216BA06AFFF743
:1096B000EDFD20B16C60002070BD092070BD082058
:1096C00070BD0000280100200E4810B50069B0B13F
:1096D0000020FCF797FC002810D1FBF78BFD08B1A8
:1096E000022000E0012000F04BF8072000F048F8CD
:1096F000054900200870FFF7BFF9002010BD0120C8
:1097000010BD0000ECB301002801002003480068F0
:1097100010B1806A002800D1002070476C0400203E
:10972000F0B4164F00220124032302251249134EE0
:10973000903F07F1040C80B101281BD1C1E900233F
:10974000C1E902250420C1E9042032603C60CCF864
:1097500000200020F0BC00F06FBB0B604B60C1E943
:1097600002350720C1E9043032603C60CCF800408B
:109770000220EFE7F0BC704708030020981914425C
:1097800070B5134C0546616F01B1884711480168F7
:10979000E1B18A691AB12846BDE87040104788785F
:1097A000012803D0022806D0012070BD2846BDE85C
:1097B0007040FFF7A9BAA06F08B9486808B1FFF771
:1097C0008BFA2846BDE87040FFF748BB002070BD0B
:1097D000ECB301006C040020014900F007B8000060
:1097E00050200040002100F001B800002DE9F34FA7
:1097F0000A2683B001284FD0FFF786FA05B0BDE8EE
:10980000F08F0A2541F61A5440F6B83B4FF0010A92
:10981000FFF7BBF8D8F80010C1F8009000205A46B6
:10982000401C9042FCD3C1F800A0002000E0401C86
:10983000A042FCD30A34F7F721FF08B9BC42E7D3B2
:10984000BC422FD219490420FFF702FD50B318483B
:1098500001A90069C06800F50050FFF749F9164CEE
:1098600014492046FFF748FD50B169462046FFF7EE
:1098700009FA28B10098800305D46D1EF5D211E0D5
:10988000009880030ED5049820B14946CDF8009089
:10989000FFF732FD0120B1E7DFF820804FF000092B
:1098A00047F230573046761EABD2A7E7000F005084
:1098B000ECB3010003005FA0F0ED00E00403002022
:1098C000884203D3904201D801207047002070479E
:1098D00010B50B4C02212069FDF7D4FAE068032192
:1098E000B0FBF1F201FB1201401CE060002905D140
:1098F0002069BDE810400121FDF7C4BA10BD000089
:10990000040100202DE9F041224D16460C4695F841
:10991000230038B1BDE8F0414FF430721EA10020A1
:10992000FBF703BBF00522D000204FF431721AA1DF
:10993000FBF7FBFA95F8210040F2C52216A1FBF7D0
:10994000F4FA31462046FEF741FF012704464FF066
:10995000000813280DD0142C17D085F824806869CE
:10996000304468612046BDE8F04100F0D5B80120E0
:10997000DBE7FEF757FE85F8218085F82370044663
:1099800085F82470FBF7F7FAE9E7002485F82470DE
:10999000E5E70000F82C00202E2E2F2E2E2F2E2E45
:1099A0002F736F757263652F6461706C696E6B2FB6
:1099B000647261672D6E2D64726F702F7666735FAF
:1099C0006D616E616765722E6300000070B51C4D9D
:1099D00006460C4695F82100002811D0002040F2E0
:1099E000852218A1FBF7A1FA601C00D0012040F2EB
:1099F000862214A1FBF799FA6868401C02D002E0A5
:109A00000120ECE76C6095F82700032801D185F868
:109A100027606868A04203D195F82700B04201D0C2
:109A2000032008E03046FEF72FFE20B945F80C4F22
:109A300001216975A975BDE8704000F06DB800009E
:109A4000F82C00202E2E2F2E2E2F2E2E2F736F75DA
:109A50007263652F6461706C696E6B2F64726167ED
:109A60002D6E2D64726F702F7666735F6D616E61FF
:109A70006765722E6300000030B4194C94F82050D2
:109A8000032D02D025683DB107E030BC40F23522FD
:109A900014A10020FBF749BA2060A068401C00D147
:109AA000A16094F82700032801D184F82730A06929
:109AB000904205D9E069904202D90AB103200CE036
:109AC000481C02D0A0688842F8D1032B03D094F838
:109AD00027009842F2D10020A26130BC00F01CB8EF
:109AE000F82C00202E2E2F2E2E2F2E2E2F736F753A
:109AF0007263652F6461706C696E6B2F647261674D
:109B00002D6E2D64726F702F7666735F6D616E615E
:109B10006765722E630000002DE9F04704461328A4
:109B200003D0142C01D0012000E000204FF43A7241
:109B300043A1FBF7FAF94F4D95F8200003280CD00C
:109B4000296891B1D5E9060282420ED368B1D5E900
:109B50000102904209D1012008E0BDE8F0474FF42E
:109B60003B7237A10020FBF7E0B9002085F8250003
:109B700095F8269019B995F82710032901D00121ED
:109B800000E00021884620B195F8241009B1012693
:109B900000E0002695F8231011B108B1012000E083
:109BA0000020824628690027401C10D06868401CAD
:109BB00000D0012040F20A3221A1FBF7B6F9696812
:109BC0002869401A69694002814200D901270320AF
:109BD00014B185F820001DE0B9F1000F09D00FB1D4
:109BE0000624F6E7B8F1000FF3D0002EF1D10424DB
:109BF000EFE7BAF1000FECD10EB1022003E0B8F1AB
:109C0000000F03D0012085F8200012E095F8200015
:109C100003280BD195F8210030B1FEF703FD002198
:109C200085F8211004B9044613480470B9F1000FF7
:109C300003D1BDE8F04701F01BB8BDE8F087000094
:109C40002E2E2F2E2E2F2E2E2F736F757263652FB3
:109C50006461706C696E6B2F647261672D6E2D6428
:109C6000726F702F7666735F6D616E616765722EBD
:109C700063000000F82C00208C00002070B5394CE7
:109C8000394B3A4960681022394D98420AD10E6822
:109C900046F440260E6037490A60091D0A68102AFA
:109CA000FCD10CE0A8420ED10E6846F440060E60CE
:109CB000304910310A60091D0A68102AFCD1984207
:109CC00003D100210CE0002070BD2B49884201D156
:109CD000012105E0A84201D1022101E04FF0FF314E
:109CE000264B1D68DA138A4015431D60196891439D
:109CF0001960016821F0060101600021816141695C
:109D00004161016841F030010160C16821F4F8113E
:109D1000C160C168C160016841F00601016094F949
:109D20000000FBF73CF86068816821F4F81181605D
:109D3000816841F4C01181604C218161016841F06A
:109D4000010101600E494FF480542246A1F1100038
:109D5000FBF79AF90B492246A1F11000FBF794F9A1
:109D6000012070BD24030020002001404405004074
:109D700000400140300C00400030014048080040E5
:109D8000DC370020EC4700200A4601460148FBF77B
:109D9000FFB90000DC47002010B508494FF480549B
:109DA0002246A1F11000FBF76FF905492246A1F107
:109DB0001000FBF769F9012010BD0000DC3700201E
:109DC000EC47002070B51A4D00246A681460417990
:109DD00001292BD0022929D0032927D0042925D0F5
:109DE0000179052906D006290AD007290AD01029A9
:109DF0001CD030248179012906D0022906D103E044
:109E00001024F7E72024F5E744F48074C179012990
:109E10000CD002290AD00068FEF786FA6868046050
:109E2000016841F007010160012070BD002070BD94
:109E30002403002070470000094918B1022807D008
:109E4000002070470748486007488860222004E0E7
:109E50000648486006488860242008700120704742
:109E60002403002000200140003010400040014049
:109E7000005010402DE9F04105460F460C461548AC
:109E8000FBF7F3F8144E90B11BE096F90000FAF7D7
:109E900075FF7168C1F81480B16815F8010B08707E
:109EA000641EA4B296F90000FAF779FF01E04FF0C2
:109EB00004087068806800F01F00202801D2002C80
:109EC000E3D1224629460348FBF779F980B2381AD4
:109ED000BDE8F081CC370020240300200148FBF7C7
:109EE000B7B80000CC3700202DE9F04186B00F460E
:109EF000DDE90C4180461D46164602A800F032FC02
:109F000002A900220A54CDE900412B4632463946C7
:109F10004046FEF7A5FC06B0BDE8F08110B50D4C3B
:109F2000207830B100202070FAF71EFF40B11F20CA
:109F300010BD832208A10020FAF7F7FF022010BD10
:109F4000607810B9FBF764FB08B1002010BD252034
:109F500010BD0000600000202E2E2F2E2E2F2E2E42
:109F60002F736F757263652F6461706C696E6B2FF0
:109F7000647261672D6E2D64726F702F6961705FFE
:109F8000666C6173685F696E74662E630000000022
:109F90002DE9FF4107466448009015460E46002310
:109FA000384600F0CBFB044660A0009023462A46CA
:109FB00031463846FBF7B8FC044460A000902346C5
:109FC0002A4631463846FBF7AFFC0444FBF712F94A
:109FD0005EA1CDE9001023462A4631463846FEF7F9
:109FE000FDF90444FBF70EF95BA1CDE9001023460F
:109FF0002A4631463846FEF7F1F90444FBF712F9D8
:10A000005AA1CDE9001023462A4631463846FEF7CC
:10A01000E5F90444FBF7FEF859A1CDE90010234609
:10A020002A4631463846FEF7D9F90444FBF7C0F911
:10A030005BA1CDE9001023462A4631463846FEF79B
:10A04000CDF904445AA0009023462A4631463846AA
:10A0500000F074FB04445DA0009023462A4631467C
:10A060003846FBF761FC0444FCF756FBF8B15DA0F1
:10A070002346D0E90010CDE902105CA000902A46EA
:10A080003146384600F05AFB0444FCF75DFB0146BC
:10A09000042202A800F090FB062102A8CDE90001ED
:10A0A00023462A463146384600F024FB04445548EE
:10A0B000009023462A463146384600F03FFB0444D0
:10A0C000FCF72AFB58B1FCF747FB4FA1CDE9001084
:10A0D00023462A4631463846FCF792FA0444FCF7F8
:10A0E00041FB4DA1CDE9001023462A4631463846B2
:10A0F000FCF786FA4C4904444CA049682346CDE954
:10A1000000012A4631463846FFF7EEFE04444BA0D4
:10A11000009023462A4631463846FBF705FC04B03A
:10A120002044BDE8F0810000D0C00100556E697187
:10A1300075652049443A2040550D0A00484943209E
:10A1400049443A2040440D0A000000004175746FF4
:10A1500020526573657400004175746F6D61746998
:10A160006F6E20616C6C6F77656400004F7665726E
:10A17000666C6F7720646574656374696F6E000048
:10A18000496E636F6D70617469626C6520696D61A1
:10A19000676520646574656374696F6E0000000014
:10A1A000506167652065726173696E670000000029
:10A1B0004461706C696E6B204D6F64653A20496E26
:10A1C000746572666163650D0A000000496E74650E
:10A1D00072666163652056657273696F6E3A2040DE
:10A1E000560D0A00000000000D0A0000426F6F7457
:10A1F0006C6F616465722056657273696F6E3A2088
:10A200000000000094C10100426F6F746C6F6164C4
:10A210006572204352430000496E74657266616343
:10A2200065204352430000009C00002052656D6F82
:10A23000756E7420636F756E7400000055524C3A51
:10A240002040520D0A0000002DE9F04341A0404E8D
:10A25000D0E9001291B0007A31607260002430724F
:10A260000927FBF789F8DFF8F88001285ED0FBF7B3
:10A2700065FC00285AD0274688F80440012406F1DE
:10A280000905182237A16846F6F7B1F91722694681
:10A290002846F6F725F9AF70202700F073F900BFC4
:10A2A00088F800402046641C88F80140651CB146CF
:10A2B00004463E44442231496846F6F798F9422262
:10A2C00069463046F6F70CF906F8024F4237347209
:10A2D00086F82040641C86F8214086F82B40F8F769
:10A2E000A3FC88F803506C1C09EB0706202224A16C
:10A2F0006846F6F77CF9202269463046F6F7F0F812
:10A30000B570203700F0E6F825A188F80540D1E9BE
:10A31000002309EB0700097A026043600172847030
:10A320000F480A30847311B0BDE8F083B8F8060016
:10A330000749401EA8F806000871742048801B4990
:10A34000002086F87400088817380880A8E7000005
:10A35000EC57002009028B0005010080FA00000084
:10A360003403002009040000020806500807058392
:10A37000024000000705040240000000D8BD0100B3
:10A380000904000002030000060921000100012267
:10A390002100070581034000010705020340000179
:10A3A0000904000000FF0300070000003C03002038
:10A3B00002484078002800D001207047580500204E
:10A3C000F8F78CBD002070477CB51C461546012867
:10A3D0001CD10CB1012C19D101AA69460C48F7F720
:10A3E000D0F870B1019A402A05DD4E2209A1002063
:10A3F000FAF79BFD0AE028460099F6F771F840202D
:10A400007CBD012C02D10D490120087000207CBDCB
:10A41000646400202E2E2F2E2E2F2E2E2F736F755C
:10A420007263652F7573622F6869642F7573626438
:10A430005F757365725F6869642E63001C05002098
:10A440002DE9F04107461D4816460088824202DD8C
:10A450000020BDE8F0811A4800780028F9D0194C96
:10A4600001224FF00008E26000E098B16288002A03
:10A47000FBD1154D3246681C2F70F6F731F8656137
:10A48000A4F8048066801148007801280BD86D1C60
:10A4900065610BE0C4F80C80C4F81480A4F8048053
:10A4A000A4F80280D4E76088401C60800020F9F79F
:10A4B00035F8074800F807800120CAE714BC0100FE
:10A4C00059050020F8040020F458002012BC0100B7
:10A4D000300400200249012008700248F7F773B8E1
:10A4E0001C050020646400207047000038B51C463D
:10A4F0001146022812D1002C10D0087807280ED05F
:10A500006B4622460B48F6F7FAFF60B10A4C2078FA
:10A51000002803D0FCF79CF80020207038BD0749C4
:10A520000120087038BD782205A10020FAF7FDFC53
:10A5300038BD0000646400201C05002000000020DD
:10A540002E2E2F2E2E2F2E2E2F736F757263652FAA
:10A550007573622F6869642F757362645F757365C4
:10A56000725F6869642E6300054910B50020C870E9
:10A57000FFF76AFEF9F7E6FFBDE81040F9F7B6B954
:10A580005805002010B5FCF79DFC074C60600020CA
:10A59000FCF766FCE060FAF7F1FC0020607003490C
:10A5A000A070A060086010BD8C0000202405002071
:10A5B00070B514460D460646FEF7B2FE074B186806
:10A5C000002809D00120FCF7A5FA2246294630468A
:10A5D000BDE8704000F0D6BB70BD0000240500202F
:10A5E000704700002DE9F04115460E460746FEF77C
:10A5F00097FE1048006800281AD00F490F4C002021
:10A60000886094F82000032812D00120FCF782FA19
:10A610002A463146384600F053FD94F820000328BE
:10A6200006D02A4631463846BDE8F041FBF70ABA63
:10A63000BDE8F081240500208C000020F82C0020CB
:10A6400006484FF0011201780548C18000210170D1
:10A650004170C0E9022101617047000008BC01009F
:10A660005805002010B50122032808DDC00020385D
:10A6700008448240064801680A43026010BD044B4A
:10A680001B1F1C6801EBC000824014431C6010BDFE
:10A69000040D004010B5EFF3108472B6FAF728FEEF
:10A6A00084F3108810BD70B50D460446090E00F005
:10A6B00013F80646A019C5F3074100F00DF806444B
:10A6C000A019C5F3072100F007F80644E9B2A01964
:10A6D00000F002F8304470BD054A02EB111301F09E
:10A6E0000F011B780370515C41700220704700001D
:10A6F000C2B801002DE9F0411446DDE906E55FEA44
:10A70000000C18D05F19A74215D32144994212D3E7
:10A71000002006462A46A34202D2E01A121A00E09E
:10A720001E1B8F4201D9791A521A0EEB00010CEB55
:10A730000600F5F7D5FE2846BDE8F0812DE9FC417D
:10A740008046089C1D4616460F462046F5F752FEE9
:10A75000CDE900402B46324639464046FFF7CAFF56
:10A76000BDE8FC81F0B50646002002460B460A25EE
:10A7700004E0B3FBF5F3401C42F10002002BF8D1DA
:10A7800050EA020301D10120002200231F460EE0FF
:10A79000B1FBF5F405FB1414B1FBF5F13034B0EB6B
:10A7A000030CBCF1010C03F1010306F80C401C1A68
:10A7B00077EB0204ECD3F0BD2DE9F04115460E46CF
:10A7C0000746FFF7CFFF0446A8420AD230222946A7
:10A7D0003846F5F73EFF281B38443146FFF7C2FFE5
:10A7E0002846BDE8F0810000074910B5096831B17D
:10A7F000096A21B18847002800D0012010BDBDE8BA
:10A80000104000F003B800006C0400202DE9F04770
:10A810001C4906460C698CB304250027D6F8008035
:10A820008946D43406E062684046FFF749F80128BB
:10A830001FD0143421680029F5D160680028F2D1B6
:10A84000E7B116E07019D9F810400027D0F8008061
:10A850000C3406E062684046FFF732F8012807D062
:10A86000143421680029F5D160680028F2D12FB195
:10A870002D1D0C2DE6D90120BDE8F087FFE7002053
:10A88000FAE70000ECB301000B49096811B1496A0D
:10A8900001B1084701783A290AD1007A302809D055
:10A8A000322807D0332805D0342803D0352801D0EA
:10A8B00000207047012070476C0400202DE9FF5FE5
:10A8C000994692468B460098FBF7FCF840F29512A9
:10A8D0003CA1FAF72AFB48490026484DB1F80B0085
:10A8E000497B484309EB0001491EB1FBF0F7B9F180
:10A8F000000F19D00024A7F10108EE6809E0E9680B
:10A90000481C82B23E4800F0D3FCE868401C641C3E
:10A91000E8604445F3D34FF6FF723948E96800F028
:10A92000C7FCE868401CE8602869202802D34FF47F
:10A93000D5721CE03349202201EB4014401C2861F1
:10A9400031492046F5F7CCFD009801682160416847
:10A95000616001892181807AA072C4F81C90300C5A
:10A96000A0826683A968102909D34FF4DC7215A16F
:10A970000020FAF7DAFA002004B0BDE8F09F214B7E
:10A9800001EB4100C03B214A43F8202003EB800249
:10A990001F4E5660BBF1000F01D043F820B0BAF152
:10A9A000000F01D0C2F804A01348491CB0F80B30C6
:10A9B000407B43437B439360A9602878401C287008
:10A9C0002046D9E72E2E2F2E2E2F2E2E2F736F7569
:10A9D0007263652F6461706C696E6B2F647261675E
:10A9E0002D6E2D64726F702F7669727475616C5F55
:10A9F00066732E6300000000642D0020A400002078
:10AA0000642F002024320020C4B7010079770100B0
:10AA1000E9B30100C07A7047C0697047C16961B18C
:10AA2000074A084B408BB2F80B105B69527BB3FBB3
:10AA3000F1F1801E00FB021070474FF0FF307047AD
:10AA4000642D0020A4000020C17270470A4910B58F
:10AA50000846B1F81340B0F80B000CB90C6A0CB101
:10AA6000444306E0002440F2891204A12046FAF78C
:10AA70005CFA204610BD0000642D00202E2E2F2EE3
:10AA80002E2F2E2E2F736F757263652F6461706C7D
:10AA9000696E6B2F647261672D6E2D64726F702FFB
:10AAA0007669727475616C5F66732E6300000000D6
:10AAB0002DE9F0410F4680464FF4007631464F486D
:10AAC000F5F7F1FD31464E48F5F7EDFD4D4C00250B
:10AAD000C0214D48E560F5F7E6FD4B487100C030F8
:10AAE000F5F7E1FD256125704848C4E901053246C6
:10AAF000474942486561F5F77AFD404E07F58037D2
:10AB000040F62D02B6F80B00717BB7FBF0F011FB9D
:10AB100002F2B0EB420F0BD24FF4AB723DA100201A
:10AB2000FAF703FA707B41F25A0110FB01F00EE0D4
:10AB30004FF691725143814209D240F2591235A128
:10AB40000020FAF7F2F9707B4FF691714843B0F5A7
:10AB5000803F03D3A6F81350306202E0A6F813003A
:10AB60003562717B3022B0FBF1F040F2FF1101EB56
:10AB70004000C0F34F27F78233492348F5F737FDEC
:10AB8000214978024861086204206561A0600020C4
:10AB900000EB400201EB820263699268401C1A4498
:10ABA00062610428F4D34FF6F87229461448E56030
:10ABB00000F07EFBE1684FF6FF72491C1048E1602F
:10ABC00000F076FBE0682049401CC4E903050E4D07
:10ABD0002022C03528463031F5F782FCD8F8001025
:10ABE0002960D8F804106960B8F80810298198F82D
:10ABF0000A00A87201202061BDE8F081642D0020C8
:10AC0000642F0020A400002064310020735901004B
:10AC100074B501002E2E2F2E2E2F2E2E2F736F7512
:10AC20007263652F6461706C696E6B2F647261670B
:10AC30002D6E2D64726F702F7669727475616C5F02
:10AC400066732E630000000074B7010010B504465F
:10AC5000FEF794FB05493CB1887808B9022088705A
:10AC6000BDE81040FEF792BB0020F8E78C00002002
:10AC700010B5FEF783FBFAF7DFF928B904484178ED
:10AC8000022901D101218170BDE81040FEF77EBB91
:10AC90008C00002010B5FEF743FB0148007810BD82
:10ACA0008C0000202DE9F0410446FEF739FBFEF749
:10ACB00065FBFAF7C1F980B1FCF766FD214A4EF653
:10ACC00060239168994201D22144916028B194781F
:10ACD00055785470012C06D103E0BDE8F041FEF731
:10ACE00055BB0220907000269660FEF74FFB0127AF
:10ACF000CDB1012D17D0022D15D1134D95F820009F
:10AD0000032804D085F826700020FEF705FF95F88B
:10AD10002000032812D0002040F211120BA1FAF7F4
:10AD200004F900F0F5F8164D54B1012C08D0022CAE
:10AD300002D1FAF723F92F60BDE8F0810120EBE79B
:10AD40002E60F9E78C000020F82C00202E2E2F2EEC
:10AD50002E2F2E2E2F736F757263652F6461706CAA
:10AD6000696E6B2F647261672D6E2D64726F702F28
:10AD70007666735F6D616E616765722E63000000B9
:10AD8000240500202DE9F0478A4604461546002692
:10AD900051025046F5F765FCDFF84890002006EBBD
:10ADA000460209EB82018442896800EB5121884602
:10ADB0000ED38C420CD2A8EB0407AF4200D32F462F
:10ADC00059F82230201A3A46514698473C44ED1B28
:10ADD000002D04D0761CF6B24046102EDFD3BDE81D
:10ADE000F08700006431002001494860704700008E
:10ADF000A40000201CB52D4CE07F10B104F11F0011
:10AE000000E02BA04FF08061FFF752FE2B48FBF7CC
:10AE1000E7FA0346207D10B12448143000E028A052
:10AE200000222649FFF74AFD2848FBF7D9FA0346D6
:10AE30000022264926A0FFF741FDFFF72BFF40B176
:10AE40002648FBF7CDFA03460022244924A0FFF749
:10AE500035FD264B41219A1C2548FAF757FA58B17F
:10AE60002448FBF7BDFA0346002222492248FFF797
:10AE700025FD0021FFF7E8FD002001904FF4803010
:10AE80000090FAF7C7FB70B1DDE900102022F5F75A
:10AE900085FA40B91948FBF7A3FA0346002217497F
:10AEA00017A0FFF70BFD00F031F81CBDECB301005B
:10AEB0004441504C494E4B20202020009D760100FB
:10AEC0004D4245442020202048544D00B5750100D6
:10AED00044455441494C532054585400C97501000D
:10AEE0004641494C20202020545854009C0000200A
:10AEF000202D002061740100C8B401001177010009
:10AF00004E4545445F424C20545854007047000061
:10AF100010B5FAF77DFB20B1FFF7BCFE08B9F7F7D3
:10AF2000D1FCFAF777FB40B1FAF73AFA18B9FAF719
:10AF300023FA012801D1F7F7C5FC02484168491CF2
:10AF4000416010BD9C000020F8B50C46074600F09B
:10AF5000B3F8002856D1FBF76DFA10B9FBF768FA81
:10AF600000B1012018B9FAF74DF900284AD0022C97
:10AF700048D074B1012C45D10B2241493846F5F730
:10AF80000DFA00283ED1FFF785FBBDE8F840FFF73A
:10AF90006FBE01208DF80000851E6946384600F01E
:10AFA0008DF8002864D1364E00240C360B2256F85A
:10AFB00034103846F5F7F2F910B906EBC4000579FC
:10AFC000641C102CF2D3681C4FF0000418D0102D14
:10AFD00048D2DFE805F008104D182325292B2F3122
:10AFE00035373B3D4143FAF715FB002840D001209F
:10AFF000FAF718FA3CE0E22222A10020F9F795FFC7
:10B000008DF80040F8BD2B4C206800688047206810
:10B010000069804720684068804729E0012000E0FF
:10B020000020FAF749FA23E0012000E00020FAF7B7
:10B030004BFA1DE0012000E00020FAF755FA17E076
:10B04000002000E00120FAF7E7F911E0012000E01C
:10B050000020FAF741FA0BE0012000E00020FAF7A7
:10B06000E7F905E04FF4887206A10020F9F75DFFCB
:10B070009DF800000028C5D0FFF7FAFDF8BD0000DC
:10B08000C8B401002E2E2F2E2E2F2E2E2F736F754B
:10B090007263652F6461706C696E6B2F6472616797
:10B0A0002D6E2D64726F702F7666735F7573657287
:10B0B0002E630000B4B801000020704700207047E4
:10B0C0002DE9F05F0446002615468B463046DFF832
:10B0D0005090DFF850A01CE006EB460209EB82021C
:10B0E0008442916800EB512188460DD38C420BD2EB
:10B0F000A8EB0407AF4200D32F465368201A3A4604
:10B10000594698473C44ED1B002D06D0761C40461E
:10B11000F6B2DAF808108E42DED3BDE8F09F0000E8
:10B1200064310020A4000020FEB5044690F83000F1
:10B1300015460F46302801D3606B31E0C0F1300670
:10B14000AE4200D3164620443246F5F7C9F994F8CA
:10B1500030003044C1B284F83010302901D20020D0
:10B16000FEBD00233744AD1B1A462046FAF728FDE2
:10B1700008B302A90022009101AB1146FAF76EFD57
:10B180000028EDD10198606394F830202146FAF749
:10B1900073FE0028E4D194F83010606B08446063BB
:10B1A0002A463946FAF768FE0028D9D1606B284450
:10B1B00060631420FEBD1C20FEBD00002DE9F84F89
:10B1C000894681184FF48063B3EB412F07D2BDE865
:10B1D000F84F4FF41F7227A10020F9F7A6BE4102D5
:10B1E0004B0951024FEA511B00912F4901EB431AC1
:10B1F00010B100262D4F33E00126FBE709EB461482
:10B200000AEB4615202221462846F5F7C7F830B349
:10B21000214628460B22F5F7C1F878B10020804678
:10B22000D7F804C023462A4620460221E04720786A
:10B23000E52805D0B8F1000F07D010E00120EEE7B7
:10B240002A4623461046012107E02046FAF73AFC39
:10B2500028B123462A46184600217C68A047761C60
:10B260005E45CBD350464946009ABDE8F84FF5F706
:10B2700037B900002E2E2F2E2E2F2E2E2F736F75E6
:10B280007263652F6461706C696E6B2F64726167A5
:10B290002D6E2D64726F702F7669727475616C5F9C
:10B2A00066732E630000000024320020A4000020FA
:10B2B00030B44B00012404EB4101B1F5007F06D30B
:10B2C00030BC40F2391204A10020F9F72EBEC2545E
:10B2D000120A425430BC70472E2E2F2E2E2F2E2EA7
:10B2E0002F736F757263652F6461706C696E6B2F5D
:10B2F000647261672D6E2D64726F702F766972743F
:10B3000075616C5F66732E63000000002DE9F047E5
:10B3100086B0002416460F460546039404940DF1AA
:10B3200010080DF10C094FF4807A0594CDF800A0B7
:10B33000CDE901986B1C05AA31463846FBF748FE5B
:10B3400068B1022813D001281DD0042825D0052873
:10B3500001D00628EAD1052821D0012020E0049A56
:10B3600022B3691C0398FAF787FD04461EE0049A8D
:10B370002AB1691C0398FAF77FFD040016D10598DD
:10B38000361A0744D2E7049A22B1691C0398FAF7E7
:10B3900073FD044654B9132408E0152406E0002088
:10B3A0004FF4B07203A1F9F7C0FD162406B0204691
:10B3B000BDE8F0872E2E2F2E2E2F2E2E2F736F7579
:10B3C0007263652F6461706C696E6B2F6472616764
:10B3D0002D6E2D64726F702F66696C655F73747269
:10B3E00065616D2E630000007047000001000217C8
:10B3F000303432330000000001000000440100201E
:10B400004D4158373830303048544D00000000006E
:10B41000000000000000687474703A2F2F7777776F
:10B420002E6D6178696D696E7465677261746564AB
:10B430002E636F6D2F6D61783738303030667468E9
:10B44000720000000000000000000000000000008A
:10B4500000000000000000000000000000000000EC
:10B4600000000000000000000000000000000000DC
:10B47000322E312E30000000396801001D9F01007E
:10B4800081720100CD56010039560100BD730100E3
:10B4900091570100999301000000000078B4010069
:10B4A00000000000FFFFFFFFFFFFFFFFFFFFFFFFA8
:10B4B000FFFFFFFF00000000000000000000000090
:10B4C0000000000000000003415353455254202067
:10B4D0005458540084B801000000000054C3010017
:10B4E0000100000060C301000200000048C3010029
:10B4F000030000003CC301000400000030C3010051
:10B5000005000000F4C201000600000018C301009D
:10B5100007000000E8C20100080000000CC30100A1
:10B5200009000000D0C201000A000000DCC20100D6
:10B530000B00000000C301000C00000024C3010048
:10B540000D0000006CC301000E00000078C3010074
:10B550000F00000090C30100ACC301009CC30100B8
:10B56000A4C3010084C30100307800000000000083
:10B5700000000000EB3C904D53443053342E31001A
:10B5800002080100022000501FF801000100010024
:10B590000000000000000000000029741902274488
:10B5A00041504C494E4B2D444E4446415431362077
:10B5B0002020FAB8C0070520018ED0BC0010B8C00A
:10B5C000078ED8BE6D00E80B00EBFEB40EB700B3DB
:10B5D00007CD10C38A044608C07405E8EDFFEBF4FC
:10B5E000C3504C454153452052454D4F564520547C
:10B5F00048452041524D204D424544204441504C45
:10B60000494E4B205553422044455649434520411D
:10B610004E44205245424F4F5420544845205359E0
:10B620005354454D2E2E0000000000000000000085
:10B63000000000000000000000000000000000000A
:10B6400000000000000000000000000000000000FA
:10B6500000000000000000000000000000000000EA
:10B6600000000000000000000000000000000000DA
:10B6700000000000000000000000000000000000CA
:10B6800000000000000000000000000000000000BA
:10B6900000000000000000000000000000000000AA
:10B6A000000000000000000000000000000000009A
:10B6B000000000000000000000000000000000008A
:10B6C000000000000000000000000000000000007A
:10B6D000000000000000000000000000000000006A
:10B6E000000000000000000000000000000000005A
:10B6F000000000000000000000000000000000004A
:10B700000000000000000000000000000000000039
:10B710000000000000000000000000000000000029
:10B720000000000000000000000000000000000019
:10B730000000000000000000000000000000000009
:10B7400000000000000000000000000000000000F9
:10B7500000000000000000000000000000000000E9
:10B7600000000000000000000000000000000000D9
:10B77000000055AA41770100E9B301000002000072
:10B7800041740100E9B301000000000041740100B0
:10B79000E9B3010000000000C1730100BDB1010068
:10B7A000000400000000000000000000000000286D
:10B7B00000000000000000000000418EBB320000CD
:10B7C0000000000000000000000000000000000178
:10B7D00000000000764876480000DC8376480000D0
:10B7E00000000000E4CA0100A0CA010080CA0100F4
:10B7F00044CB01008CC7010048CA0100A4C7010066
:10B8000060C90100B8C9010000CB01000CCA0100E9
:10B8100014C9010038C9010084C90100B8CA010077
:10B8200040C8010014C80100ECC7010070C8010045
:10B83000ECC9010028CB010020C50100E0C40100D3
:10B84000A4C40100A0C801001CC7010078C6010003
:10B8500040C6010068C5010050C7010044C4010092
:10B8600078C4010018C40100B8C30100E8C3010096
:10B87000D8C60100B8C50100F4C501006CCB0100B9
:10B88000B4C6010053544152545F424C41435400EA
:10B8900005950100C99601005595010035940100F8
:10B8A000B99301006196010091940100A9930100F0
:10B8B0008D96010090B80100000000000000010119
:10B8C00001003031323334353637383961626364E0
:10B8D0006566000000BE0AE00D782D066840082469
:10B8E000400000D35840641EFAD1491C521E002A61
:10B8F000F2D1704710B503460C469348484441685E
:10B90000886800F0807008B1012010BD8E4848445E
:10B91000806848600020F8E702468B484844416848
:10B92000886820F07040886000207047864848444E
:10B930004168886800F0807008B101207047486A4B
:10B9400048B100204862486A28B102204862486A2B
:10B9500008B10120F2E7886820F0704040F0005004
:10B9600088600020EAE710B5774848444468FFF74C
:10B97000DDFF08B1012010BDA06820F47F4040F435
:10B980002A40A060A06840F00200A06000BFA0684C
:10B9900000F080700028FAD1A06820F07040A0600C
:10B9A000606A00F0020008B10120E4E70020E2E74D
:10B9B00070B50546644848444468FFF7B7FF08B1CE
:10B9C000012070BDA06820F47F4040F4AA40A06030
:10B9D0002560A06840F00400A06000BFA06800F0EF
:10B9E00080700028FAD1A06820F07040A060606AE2
:10B9F00000F0020008B10120E3E70020E1E72DE9B3
:10BA0000F04707468A4690464F48484444685646A1
:10BA1000454608F0030010B10120BDE8F087454617
:10BA2000FFF784FF08B10120F7E7A06820F000606D
:10BA3000A060A06840F01000A0600EE0276001CD7B
:10BA40002063A06840F00100A06000BFA06800F083
:10BA500080700028FAD13F1D361F042E03D307F053
:10BA60001F000028EAD138484844C068802821D106
:10BA7000102E1FD3A06820F01000A060A06840F036
:10BA80000060A06014E0276001CD206301CD6063F9
:10BA900001CDA06301CDE063A06840F00100A0608B
:10BAA00000BFA06800F080700028FAD11037103E67
:10BAB000102EE8D2042E19D3A06820F00060A060F8
:10BAC000A06840F01000A0600EE0276001CD206368
:10BAD000A06840F00100A06000BFA06800F0807086
:10BAE0000028FAD13F1D361F042EEED206B3A268FD
:10BAF00022F00062A260A26842F01002A2604FF041
:10BB0000FF30FF2105E02A6862EA010210400902C5
:10BB1000761E002EF7D127602063A26842F0010252
:10BB2000A26000BFA26802F08072002AFAD100BFB2
:10BB3000A06820F07040A060606A00F0020008B1C8
:10BB400001206AE7002068E7040000000000000010
:10BB5000000000000090024064000000800000002F
:10BB6000000000100000080000200000000000108D
:10BB7000002000002100002045000020930000204C
:10BB8000DD0000202B01002000000000010000204B
:10BB90007802002000100020000400200000002097
:10BBA00098020000D4B8010000020000000000006C
:10BBB000011701000000000000000000000000006C
:10BBC0000000000000000000D99701000000000004
:10BBD000000000000000000000000000021701004B
:10BBE0000000000000000000000000000000000055
:10BBF00000000000E59701000000000000000000C8
:10BC000000000000000000000000014001024000B0
:10BC100040000101400040000304400000024000D9
:10BC200006074000400040004000212000000000C6
:10BC3000514C010000000000000000000130010034
:10BC40001D35010065360100F93B0100FD3B010097
:10BC5000E52B01007D2A0100492B010000000000B6
:10BC600000000000000000000000000000000000D4
:10BC7000000000000000000000000000D92E0100BC
:10BC800000000000000000000600FF0901A10115EE
:10BC90000026FF00750895400901810295400901C1
:10BCA000910295010901B102C000210012011002A8
:10BCB000EF020140280D0402001001020301000000
:10BCC000050F3900021810050038B60834A909A07C
:10BCD000478BFDA0768815B665000121001C100574
:10BCE00000DF60DDD88945C74C9CD2659D9E648A83
:10BCF0009F00000306AA00200000040309040803B3
:10BD0000410072006D0024034400410050004C00CB
:10BD100069006E006B00200043004D005300490095
:10BD200053002D004400410050001A033000300041
:10BD30003000310041003000300030003000300071
:10BD40003000300022036D006200650064002000B6
:10BD5000530065007200690061006C002000500013
:10BD60006F007200740022036D00620065006400C1
:10BD70002000530065007200690061006C00200023
:10BD800050006F00720074001A0343004D0053000E
:10BD9000490053002D00440041005000200076006F
:10BDA0003100240357006500620055005300420033
:10BDB0003A00200043004D005300490053002D007D
:10BDC00044004100500010035500530042005F0042
:10BDD0004D00530043000000080B00020202010462
:10BDE00009040000010202010405240010010524D9
:10BDF000010302042402060524060000070585034A
:10BE000010002009040000020A00000507050702CF
:10BE1000400000070586024000000400880004017D
:10BE2000FFA50E0001000000102700000000000028
:10BE3000CC00000098000000040000000100010098
:10BE400000000000000000000000000000000000F2
:10BE500000000000000000000000000000000000E2
:10BE600000000000000000000200020001000000CD
:10BE700000000000000000000000000000000000C2
:10BE800000000000000000000000000000000000B2
:10BE90000000000003000200040000000000000099
:10BEA0000000000000000000000000000000000092
:10BEB0000000000000000000000000000000000082
:10BEC0000000000000000000000000000000000072
:10BED0000000000000000000000000000000000062
:10C0D00023204441504C696E6B204669726D776134
:10C0E0007265202D207365652068747470733A2F13
:10C0F0002F6461706C696E6B2E696F0D0A427569F1
:10C100006C642049443A2076303235382D626574AB
:10C1100061332D6730303034313938622028617214
:10C120006D6363290D0A00004120626F6F746C6FAC
:10C130006164657220757064617465207761732035
:10C14000737461727465642062757420756E6162C7
:10C150006C6520746F20636F6D706C6574652E0D57
:10C160000A52656C6F61642074686520626F6F7439
:10C170006C6F6164657220746F20666978207468E2
:10C180006973206572726F72206D65737361676584
:10C190002E0D0A00476974205348413A2030303050
:10C1A000343139386233616439623039333861315E
:10C1B0003033396532383430356237353966656148
:10C1C00037386331310D0A4C6F63616C204D6F64F9
:10C1D000733A20300D0A55534220496E74657266D9
:10C1E000616365733A204D53442C204344432C2013
:10C1F0004849442C205765625553420D0A000000FF
:10C200003C21646F63747970652068746D6C3E0DB9
:10C210000A3C212D2D206D62656420506C6174668E
:10C220006F726D205765627369746520616E64205A
:10C2300041757468656E7469636174696F6E2053CB
:10C24000686F7274637574202D2D3E0D0A3C6874FE
:10C250006D6C3E0D0A3C686561643E0D0A3C6D657F
:10C26000746120636861727365743D227574662D14
:10C2700038223E0D0A3C7469746C653E6D626564DB
:10C2800020576562736974652053686F72746375B3
:10C29000743C2F7469746C653E0D0A3C2F686561AF
:10C2A000643E0D0A3C626F64793E0D0A3C73637212
:10C2B0006970743E0D0A77696E646F772E6C6F63D8
:10C2C0006174696F6E2E7265706C616365282200FF
:10C2D0004D53445F4F4E2020434647004D53445F2B
:10C2E0004F464620434647004F56464C5F4F4E2030
:10C2F000434647004155544F5F4F4E204346470049
:10C30000434F4D505F4F4E20434647004F56464CDB
:10C310005F4F4646434647004155544F5F4F4646A0
:10C3200043464700434F4D505F4F46464346470004
:10C33000484152445F525354434647004155544F7D
:10C340005F525354434647004552415345202020F5
:10C35000414354004153534552542020414354001B
:10C3600052454652455348204143540050414745A9
:10C370005F4F4E2041435400504147455F4F464672
:10C3800041435400696E7465726661636500000024
:10C39000696E7465726E616C000000007573657281
:10C3A0000000000074617267657400007472616E51
:10C3B0007369656E74000000496E206170706C696D
:10C3C000636174696F6E2070726F6772616D6D6901
:10C3D0006E6720736563746F722065726173652088
:10C3E0006661696C65642E00496E206170706C69CD
:10C3F000636174696F6E2070726F6772616D6D69D1
:10C400006E67206D6173732065726173652066616C
:10C41000696C65642E000000496E206170706C6963
:10C42000636174696F6E2070726F6772616D6D69A0
:10C430006E67207772697465206661696C65642E29
:10C4400000000000496E206170706C69636174695E
:10C450006F6E2070726F6772616D6D696E672069B3
:10C460006E697469616C697A6174696F6E20666166
:10C47000696C65642E000000496E206170706C6903
:10C48000636174696F6E2070726F6772616D6D6940
:10C490006E6720756E696E6974206661696C65648B
:10C4A0002E000000546865206865782066696C6518
:10C4B0002063616E6E6F742062652070726F6772A8
:10C4C000616D6D65642E204C6F67696320666169DC
:10C4D0006C757265206F636375727265642E0000FF
:10C4E000546865206865782066696C652063616EB4
:10C4F0006E6F74206265206465636F6465642E20CE
:10C50000506172736572206C6F6769632066616940
:10C510006C757265206F636375727265642E0000BE
:10C52000546865206865782066696C652063616E73
:10C530006E6F74206265206465636F6465642E208D
:10C54000436865636B73756D2063616C63756C61C3
:10C5500074696F6E206661696C757265206F6363C4
:10C5600075727265642E0000546865206170706C8D
:10C5700069636174696F6E2066696C6520666F72AD
:10C580006D617420697320756E6B6E6F776E2061BC
:10C590006E642063616E6E6F7420626520706172DC
:10C5A00073656420616E642F6F722070726F6365B3
:10C5B000737365642E000000496E206170706C69B1
:10C5C000636174696F6E2070726F6772616D6D69FF
:10C5D0006E67206E6F7420737570706F727465640F
:10C5E000206F6E2074686973206465766963652EB8
:10C5F00000000000496E206170706C6963617469AD
:10C600006F6E2070726F6772616D6D696E67206604
:10C6100061696C6564206265636175736520746827
:10C6200065207570646174652073656E7420776130
:10C630007320696E636F6D706C6574652E00000009
:10C64000546865207374617274696E6720616464F4
:10C650007265737320666F722074686520696E74EA
:10C6600065726661636520757064617465206973C5
:10C670002077726F6E672E00546865207374617244
:10C6800074696E67206164647265737320666F728B
:10C690002074686520626F6F746C6F6164657220CE
:10C6A0007570646174652069732077726F6E672E90
:10C6B0000000000054686520626F6F746C6F6164E5
:10C6C00065722043524320646964206E6F74207049
:10C6D0006173732E00000000496E206170706C69F8
:10C6E000636174696F6E2070726F6772616D6D69DE
:10C6F0006E672061626F7274656420647565207472
:10C700006F20616E206F7574206F6620626F756E8A
:10C71000647320616464726573732E0054686520CD
:10C720006865782066696C65206F6666736574203D
:10C730006C6F616420616464726573732069732037
:10C740006E6F7420636F72726563742E0000000058
:10C75000546865206170706C69636174696F6E20E4
:10C76000696D616765206973206E6F7420636F6DFA
:10C7700070617469626C652077697468207468659B
:10C78000207461726765742E000000005468652093
:10C790007472616E736665722074696D6564206F72
:10C7A00075742E0046696C652073656E74206F7514
:10C7B00074206F66206F7264657220627920504326
:10C7C0002E20546172676574206D69676874206EED
:10C7D0006F742062652070726F6772616D6D656441
:10C7E00020636F72726563746C792E00466C61739E
:10C7F0006820616C676F726974686D207772697404
:10C800006520636F6D6D616E64204641494C5552E1
:10C8100045000000466C61736820616C676F726947
:10C8200074686D20657261736520616C6C20636F44
:10C830006D6D616E64204641494C555245000000C3
:10C84000466C61736820616C676F726974686D20F3
:10C85000657261736520736563746F7220636F6DB9
:10C860006D616E64204641494C5552450000000000
:10C87000466C61736820616C676F726974686D20C3
:10C8800077726974652076657269667920636F6D69
:10C890006D616E64204641494C55524500000000D0
:10C8A000546865206865782066696C6520796F75C5
:10C8B0002064726F707065642069736E27742063E2
:10C8C0006F6D70617469626C65207769746820743B
:10C8D000686973206D6F6465206F72206465766986
:10C8E00063652E2041726520796F7520696E204D39
:10C8F00041494E54454E414E4345206D6F64653F5E
:10C90000205365652048454C50204641512E4854DF
:10C910004D0000004661696C656420746F20696E8B
:10C92000697469616C697A652074686520746172E4
:10C93000676574204D4355004661696C65642074D9
:10C940006F20756E696E697469616C697A652074AF
:10C95000686520746172676574204D43550000005E
:10C960004661696C656420746F2072657365742F0D
:10C9700068616C74207468652074617267657420E6
:10C980004D43550050726F6772616D6D696E67201F
:10C9900061626F727465643A20696D6167652077C2
:10C9A0006F756C64206C6F636B2074617267657463
:10C9B000204D4355000000004661696C6564207499
:10C9C0006F20646F776E6C6F616420666C61736852
:10C9D00020616C676F726974686D20746F20746178
:10C9E00072676574204D435500000000456E642059
:10C9F0006F662073747265616D2068617320626573
:10CA0000656E207265616368656400004661696CEB
:10CA1000656420746F20646F776E6C6F616420743E
:10CA2000686520666C617368206461746120636F5F
:10CA30006E74656E747320746F2062652070726FFF
:10CA40006772616D6D656400506F737369626C65C8
:10CA5000206D69736D6174636820626574776565C4
:10CA60006E2066696C652073697A6520616E64204A
:10CA700073697A652070726F6772616D6D656400AD
:10CA8000416E20696E7465726E616C206572726FA2
:10CA90007220686173206F63637572726564000051
:10CAA000416E206572726F7220686173206F6363DC
:10CAB00075727265640000004661696C656420747B
:10CAC0006F20756E6C6F636B207461726765742084
:10CAD0004D435520666F722070726F6772616D6D85
:10CAE000696E67004F7065726174696F6E2077615F
:10CAF00073207375636365737366756C0000000063
:10CB0000466C61736820616C676F726974686D2030
:10CB10006D697373696E6720666F7220612072653C
:10CB200067696F6E00000000456E64206F662073B9
:10CB3000747265616D20697320756E6B6E6F776EB0
:10CB400000000000416E206572726F72206F636397
:10CB5000757272656420647572696E6720746865A9
:10CB6000207472616E736665720000000000000040
:10CB70004D4245442020202056465320202020208E
:10CB80002020202020202020302E3100ACCB01009E
:10CB9000000000207C0500004C01010000CD0100D8
:10CBA0007C0500208C620000A8010100011014190E
:10CBB000560114056E011429B10114ED51011A2B0F
:10CBC000101A0910140DB3011AF110018D38080163
:10CBD000010206020208013A04063F0101060606A8
:10CBE00004017A10010D1F069996974A0911DB027C
:10CBF0002B04146CBB01594322106B08104F1A749C
:10CC00001801B722201A020401FF05156CDC02325C
:10CC10001205126B520A140306AA1208320212A05D
:10CC200012141203A757494E55534212841204128C
:10CC300007122A12441265127612691A6308124901
:10CC4000126E1A7408127212663A611212471A555D
:10CC500016124432731250127B12391232124312DE
:10CC60004512361A340412321A2D1212431A3702A0
:10CC70003A2D121A461C29141A33021A420A123388
:10CC80001A31203A422612351A4102291812395215
:10CC90007D1470CB0140292C03016F732E6D6265EA
:10CCA000642E636F6D2F7765627573622F6C616E92
:10CCB00064696E672D706167652F3F6269643DCA64
:10CCC000132C0149143CBE011A68041A94041AC0BA
:10CCD000041AEC041418BF011A9C041A44041A70B4
:10CCE000041AC8041AF4041420C0011A4C041A7857
:10CCF000041AA40414B0BB011ADC041AFF0101C415
:10CD0000FFFFFFFFFFFFFFFFFFFFFFFFFFFFFFFF33
:10CD1000FFFFFFFFFFFFFFFFFFFFFFFFFFFFFFFF23
:10CD2000FFFFFFFFFFFFFFFFFFFFFFFFFFFFFFFF13
:10CD3000FFFFFFFFFFFFFFFFFFFFFFFFFFFFFFFF03
:020000040007F3
:10DFF000FFFFFFFFFFFFFFFFFFFFFFFFAB348518B1
:0400000500010110E5
:00000001FF
